:020000020000FC
:100000000C94B24A18951895189518951895189546
:100010001895189518951895189518951895189578
:100020001895189518951895189518951895189568
:100030001895189518951895189518950C94A22E42
:1000400018951895189518950C9444461895189578
:100050001895189518951895189518951895189538
:100060001895189518951895189518951895189528
:1000700018951895189518950C941E46189518956E
:100080001895189518951895189518950D0A20002B
:100090000D0A0A205B434D2D352056657273696F3A
:1000A0006E20312E30365D000D0A20546F737320A0
:1000B0004D6F64650D0A000D0A202D3E5B44796E7C
:1000C000616D6978656C5D3A000D0A203C2D5B44DA
:1000D000796E616D6978656C5D3A000D0A203C2D82
:1000E0003E50433A00203C2D3E44796E616D697864
:1000F000656C3A000D0A2041726520796F75207396
:10010000757265203F28792F4E29000D0A205573FE
:10011000616765203A20476F205B506F736974698F
:100120006F6E20416E676C6528307830307E307895
:10013000336666295D000D0A20416C6C2044796E9F
:10014000616D6978656C27732049442077696C6C10
:100150002062652073657420746F20002E20417228
:100160006520796F7520737572653F28592F4E2968
:10017000000D0A204572726F72315B436865636BD4
:100180002044796E616D6978656C2056657273697B
:100190006F6E206973206D6F7265207468616E20C8
:1001A000335D000D0A2042284265666F7265292C76
:1001B0004E284E657874292C512851756974290090
:1001C0000D0A203438354D6F6E69746F72205B4CA8
:1001D000462C43522061726520616464656420612D
:1001E000742070617573652074696D655D0D0A001A
:1001F0000D0A204E6F20446174615B61742042726D
:100200006F61646361737420494420307846455DB2
:10021000000D0A204E6F20446174612843686563B5
:100220006B2049442C204F7065726174696E6720A1
:100230004D6F64652C20426175642072617465297C
:1002400000204C454E3A000D0A204C454420426C9B
:10025000696E6B2049443A002044796E616D69787B
:10026000656C7320466F756E642E000D0A204C4538
:100270004420426C696E6B2049443A000D20466F61
:10028000756E642120424155445F5245473A002C27
:100290002049443A000D0A20426175642052656786
:1002A000206973206368616E67656420746F200045
:1002B000425053000D0A2049443A30202D20000DB1
:1002C0000A2044656C61793A000D0A20546F7271FE
:1002D000756520456E61626C65000D0A204D6F7674
:1002E000652030203C2D3E203078336666000D0AB4
:1002F00020416E79204B657920746F20436F6E74B6
:10030000696E75652E2E2E000D0A205B45455052F4
:100310004F4D20415245415D0D0A204D4F44454C03
:100320005F4E554D4245525F4C202020202020201A
:1003300020285229205B000D0A204D4F44454C5F78
:100340004E554D4245525F4820202020202020203D
:10035000285229205B000D0A2056455253494F4E22
:100360002020202020202020202020202020202885
:100370005229205B000D0A20494420202020202003
:100380002020202020202020202020202028522F24
:1003900057295B000D0A20424155445F52415445A4
:1003A00020202020202020202020202028522F57CD
:1003B000295B000D0A2052455455524E5F44454C6E
:1003C00041595F54494D452020202028522F57295C
:1003D0005B000D0A2043575F414E474C455F4C4937
:1003E0004D49545F4C202020202028522F57295B54
:1003F000000D0A2043575F414E474C455F4C494D25
:1004000049545F48202020202028522F57295B0084
:100410000D0A204343575F414E474C455F4C494DC1
:1004200049545F4C2020202028522F57295B000D73
:100430000A204343575F414E474C455F4C494D4965
:10044000545F482020202028522F57295B000D0A96
:10045000202852455345525645442920202020202B
:1004600020202020202028522F57295B000D0A2011
:100470004C494D49545F54454D5045524154555295
:10048000452020202028522F57295B000D0A2044A8
:100490004F574E5F4C494D49545F564F4C5441475E
:1004A0004520202028522F57295B000D0A20555047
:1004B0005F4C494D49545F564F4C544147452020AD
:1004C00020202028522F57295B000D0A204D41582B
:1004D0005F544F525155455F4C2020202020202052
:1004E000202028522F57295B000D0A204D41585FCC
:1004F000544F525155455F48202020202020202075
:100500002028522F57295B000D0A2052455455527E
:100510004E5F4C4556454C20202020202020202096
:1005200028522F57295B000D0A20414C41524D5F44
:100530004C4544202020202020202020202020283E
:10054000522F57295B000D0A20414C41524D5F53F9
:10055000485554444F574E20202020202020285218
:100560002F57295B000D0A20285245534552564506
:100570004429202020202020202020202028522F05
:1005800057295B000D0A20444F574E5F43414C49A9
:1005900042524154494F4E5F4C20202028522F5741
:1005A000295B000D0A20444F574E5F43414C49429E
:1005B000524154494F4E5F4820202028522F57293E
:1005C0005B000D0A2055505F43414C494252415453
:1005D000494F4E5F4C202020202028522F57295B66
:1005E000000D0A2055505F43414C49425241544945
:1005F0004F4E5F48202020202028522F57295B0093
:100600000D0A205B52414D20415245415D0D0A20AB
:10061000544F525155455F454E41424C4520202094
:10062000202020202028522F57295B000D0A204C23
:100630004544202020202020202020202020202071
:100640002020202028522F57295B000D0A204357D5
:100650005F434F4D504C49414E43455F4D415247DA
:10066000494E2028522F57295B000D0A204343573B
:100670005F434F4D504C49414E43455F4D415247BA
:10068000494E28522F57295B000D0A2043575F43DC
:100690004F4D504C49414E43455F534C4F504520C0
:1006A0002028522F57295B000D0A204343575F43F0
:1006B0004F4D504C49414E43455F534C4F504520A0
:1006C00028522F57295B000D0A20474F414C5F509D
:1006D0004F534954494F4E5F4C2020202020202862
:1006E000522F57295B000D0A20474F414C5F504F56
:1006F000534954494F4E5F48202020202020285243
:100700002F57295B000D0A204D4F56494E475F5326
:10071000504545445F4C2020202020202028522F87
:1007200057295B000D0A204D4F56494E475F5350E5
:100730004545445F482020202020202028522F5764
:10074000295B000D0A20544F525155455F4C494DCD
:1007500049545F4C2020202020202028522F572948
:100760005B000D0A20544F525155455F4C494D498D
:10077000545F482020202020202028522F57295B1A
:10078000000D0A2050524553454E545F504F534977
:1007900054494F4E5F4C20202020285229205B00D6
:1007A0000D0A2050524553454E545F504F53495403
:1007B000494F4E5F4820202020285229205B000D01
:1007C0000A2050524553454E545F53504545445FAF
:1007D0004C20202020202020285229205B000D0AB8
:1007E0002050524553454E545F53504545445F4851
:1007F00020202020202020285229205B000D0A20C4
:1008000050524553454E545F4C4F41445F4C20205D
:10081000202020202020285229205B000D0A205073
:10082000524553454E545F4C4F41445F4820202071
:100830002020202020285229205B000D0A20505221
:100840004553454E545F564F4C5441474520202058
:1008500020202020285229205B000D0A20505245DC
:1008600053454E545F54454D5045524154555245A1
:10087000202020285229205B000D0A20524547499C
:100880005354455245445F494E53545255432E20CC
:100890002028522F57295B000D0A205245534552FC
:1008A0005645442850415553455F54494D452920EC
:1008B00028522F57295B000D0A204D4F56494E47AD
:1008C0002020202020202020202020202020202028
:1008D000285229205B000D0A204C4F434B2020203A
:1008E00020202020202020202020202020202852CE
:1008F0002F57295B000D0A2050554E43485F4C206E
:100900002020202020202020202020202028522F9E
:1009100057295B000D0A2050554E43485F48202060
:1009200020202020202020202020202028522F5747
:10093000295B000D0A0A2044554D50284429203ACD
:100940002044756D7020636F6E74726F6C207461DB
:10095000626C652E000D0A204944205B49445F4EBD
:10096000554D5D203A20536574204944206F662020
:1009700064796E616D6978656C2E000D0A204349BB
:1009800044205B49445F4E554D5D203A20436861E9
:100990006E676520436F6E74726F6C2049442E0041
:1009A0000D0A2052454144205B414444525D5B4C5A
:1009B000454E5D203A205265616420646174612E69
:1009C0002065782952656164203130203220285218
:1009D0006561642066726F6D20307831302C206C38
:1009E000656E677468203229000D0A2057524954F9
:1009F00045205B414444525D5B44415441315D2E8E
:100A00002E203A20577269746520646174612E202B
:100A100065782957726974652031342C3120285744
:100A20007269746520312061742030783134290076
:100A30000D0A205245475F5752205B414444525DA6
:100A40005B44415441315D2E2E203A205265676946
:100A50007374657220777269746520696E7374753A
:100A6000726374696F6E000D0A20414354494F4E02
:100A7000203A20416374696F6E205245475F575298
:100A800020696E737472756374696F6E000D0A204D
:100A9000476F205B504F534954494F4E5D5B535055
:100AA0004545445D3A20476F746F20746865207037
:100AB0006F736974696F6E207769746820746865F4
:100AC0002073706565642E000D0A20484558205B30
:100AD0004E554D5D5B4E554D5D2E2E2E203A2054C9
:100AE00072616E736D6974652072617720646174E0
:100AF000612E2065782948657820464620464620A4
:100B00003031203033000D0A205245534554203AED
:100B10002044796E616D6978656C205265736574E7
:100B20002E000D0A2050494E47205B4E554D5D3A30
:100B3000206578292050696E67204E554D20494424
:100B40002064796E616D6978656C2E000D0A205302
:100B50005752205B414444525D5B4C454E5D5B49BE
:100B6000445D5B444154415D2E2E2E5B49445D5BE8
:100B7000444154415D2E2E2E203A2053796E63203D
:100B800057726974652E000D0A205343414E205B55
:100B90004E554D5D203A205343414E206C696E6B9B
:100BA00065642064796E616D6978656C20696E207A
:100BB000307E4E554D20696E2063757272656E747D
:100BC000206261756420726174652E000D0A204CEC
:100BD0004544205B4E554D5D203A20426C696E6B5A
:100BE000204C4544206F66204E554D2049442E2010
:100BF0002742272C274E2720666F72204944206306
:100C000068616E67652E2027512720666F7220511C
:100C10007569742E000D0A2042415544205B4E55E3
:100C20004D5D203A205365742062617564207261C5
:100C300074652020657829204241554420323228AD
:100C40003537363030425053292C2042415544200C
:100C50003128314D42505329000D0A20534541524D
:100C60004348203A205365617263682049442061FB
:100C70006E64206261756472617465206F662061C4
:100C80006C6C206C696E6B65642064796E616D6953
:100C900078656C732E000D0A2055706461746520B0
:100CA0005B53544152545F49445D205B454E445F61
:100CB00049445D203A2044796E616D6978656C2005
:100CC0006669726D77617265207570646174652EF6
:100CD0002873797374656D2075736572206F6E6CFF
:100CE0007929000D0A0A2020202020202020436F8F
:100CF0007079726967687420524F424F544953208B
:100D0000434F2E2C4C54442E0D0A005B496E7661E5
:100D10006C6964205061676520526561643A000D1A
:100D20000A205B4572723A5278442054696D656FAF
:100D300075745D000D0A205B4572723A57726F6ED2
:100D400067204865616465725D000D0A205B45722D
:100D5000723A5478494420213D20527849445D003C
:100D60000D0A205B4572723A57726F6E67204C65B0
:100D70006E6774685D000D0A205B4572723A5772A7
:100D80006F6E6720436865636B53756D5D000D0A78
:100D900020555044415445205B53544152542049FE
:100DA000445D205B454E442049445D005D3A000DA2
:100DB0000A2049443A00205374616E6462792E001F
:100DC0002057726974696E672E2E00205375636315
:100DD0006573732E00204572726F722E000D0A200B
:100DE0004572722049443A002042616420436F6D8D
:100DF0006D616E64005B457869745D000D0A204D7D
:100E00004F54494F4E20504C4159205041474520A6
:100E100020202028522F5729000D0A204F4E205005
:100E20004C4159494E47204D4F54494F4E202020A8
:100E30002028522920000D0A205458205749524595
:100E40004C455353205041434B4554202028522FAA
:100E50005729000D0A20525820574952454C4553F6
:100E600053205041434B4554202020285229200034
:100E70000D0A204E4557205041434B4554204152C6
:100E8000524956454420202028522920000D0A208E
:100E9000415558204C45442020202020202020204F
:100EA0002020202028522F5729000D0A2042555477
:100EB000544F4E282D532D552D442D4C2D52292065
:100EC000202028522920000D0A2054494D4552283F
:100ED0003132356D5365632045616368292028529E
:100EE0002F5729000D0A205A4947424545204944B9
:100EF000202020202020202020202028522F572969
:100F0000000D0A20524F424F5420494420202020F7
:100F1000202020202020202028522F5729000D4457
:100F2000796E616D6978656C2020302830783030BA
:100F3000295B202020205D000D0A44796E616D69D7
:100F400078656C2020312830783031295B202020D2
:100F5000205D0020506167654E756D6265723A00D4
:100F60000D0A44796E616D6978656C2020322830F5
:100F7000783032295B202020205D0020416464729B
:100F80003A000D0A44796E616D6978656C202033F2
:100F90002830783033295B202020205D0020285223
:100FA0006573657276656429203A000D0A44796E8E
:100FB000616D6978656C2020342830783034295B85
:100FC000202020205D00202020506C6179436F7527
:100FD0006E743A000D0A44796E616D6978656C2013
:100FE00020352830783035295B202020205D0020F6
:100FF00028526573657276656429203A000D0A44AB
:10100000796E616D6978656C2020362830783036CD
:10101000295B202020205D002028526573657276B0
:10102000656429203A000D0A44796E616D6978651E
:101030006C2020372830783037295B202020205D35
:10104000002028526573657276656429203A000D88
:101050000A44796E616D6978656C20203828307893
:101060003038295B202020205D00202852657365E0
:101070007276656429203A000D0A44796E616D69C3
:1010800078656C2020392830783039295B20202081
:10109000205D002020205061676520537465703A00
:1010A000000D0A44796E616D6978656C20313028D5
:1010B00030783041295B202020205D0020436F6E76
:1010C00074726F6C436F64653A000D0A44796E6107
:1010D0006D6978656C2031312830783042295B2089
:1010E0002020205D002020506167652053706565D9
:1010F000643A000D0A44796E616D6978656C20313F
:10110000322830783043295B202020205D002020C9
:101110002044584C2053657475703A000D0A447988
:101120006E616D6978656C203133283078304429E0
:101130005B202020205D002020416363656C2054EB
:10114000696D653A000D0A44796E616D6978656C68
:101150002031342830783045295B202020205D0064
:101160004C696E6B20746F204E6578743A000D0ADE
:1011700044796E616D6978656C203135283078303E
:1011800046295B202020205D004C696E6B20746F27
:1011900020457869743A000D0A44796E616D69786A
:1011A000656C2031362830783130295B20202020B2
:1011B0005D002852657365727665645031293A0086
:1011C0000D0A44796E616D6978656C20313728307D
:1011D000783131295B202020205D0028526573651D
:1011E000727665645231293A000D0A44796E616D58
:1011F0006978656C2031382830783132295B2020BD
:1012000020205D002852657365727665645032292E
:101210003A000D0A44796E616D6978656C20313948
:101220002830783133295B202020205D002852654A
:101230007365727665645232293A000D0A44796EFC
:10124000616D6978656C2032302830783134295BE3
:10125000202020205D000D0A44796E616D6978655B
:101260006C2032312830783135295B202020205DF8
:10127000000D0A44796E616D6978656C2032322800
:1012800030783136295B202020205D000D0A44791A
:101290006E616D6978656C2032332830783137297A
:1012A0005B202020205D000D0A44796E616D697815
:1012B000656C2032342830783138295B202020209A
:1012C0005D000D0A44796E616D6978656C20323578
:1012D0002830783139295B202020205D000D0A4418
:1012E000796E616D6978656C2032362830783161AD
:1012F000295B202020205D000D0A44796E616D6914
:1013000078656C2032372830783162295B202020C4
:10131000205D000D0A44796E616D6978656C20323C
:10132000382830783163295B202020205D000D0AA9
:1013300044796E616D6978656C2032392830783176
:1013400064295B202020205D000D0A44796E616DC8
:101350006978656C2033302830783165295B20202E
:1013600020205D000D0A20202050617573655469AE
:101370006D65202020202020205B2020205D000D96
:101380000A20202053706565642020202020202022
:10139000202020205B2020205D20202020202020D5
:1013A000202020202020202020202020202020203D
:1013B000202020202020202020202020205B583AA0
:1013C0002D2D2C593A2D2D2C413A2D2D2D2D5D00F2
:1013D0000D0A202020202020202020202020202036
:1013E00020202020205354503720205354503020A8
:1013F00053545031205354503220535450332053BF
:10140000545034205354503520535450362020200B
:1014100020476F20537465703A2020202020000D53
:101420000A202020202020202020202020202020D2
:10143000202020202020202020204D5354522053B3
:101440004C4156204F46535420202020202020205D
:10145000202020202020202020202020202020208C
:10146000476F20537465703A2020202020000D0A19
:101470005D205F20202020202020202020202020F0
:10148000202020202020202020202020202020205C
:10149000202020202020202020202020202020204C
:1014A000202020202020202020202020202020203C
:1014B00020202020202020202020202000204172D9
:1014C0006520796F7520737572653F5B792F4E5D6E
:1014D0000020496E76616C69642050616765002068
:1014E000496E76616C696420506172616D657465E6
:1014F0007200204F66667365742055706461746570
:101500006400204F7574206F662052616E6765001D
:10151000204F4B000D0A20202020202020202D438A
:101520004D3A2052503D2850617261302C4F502C62
:10153000506172613129204C4B205253205B414451
:1015400044525D2020000D0A20427265616B2061CB
:101550007420000D0A204552524F523A004946204D
:101560002020202000454C534520494600454C533F
:101570004520202000616E642F6F7220004A554D77
:1015800050202020004C4F414420202000434F4D4C
:1015900050555445005354415254202000454E4468
:1015A000202020200043414C4C2020200052455454
:1015B00055524E20004E554C4C202020000D0A2044
:1015C0004845584120444953504C4159204D4F44BF
:1015D00045000D0A20444543494D414C20444953A0
:1015E000504C4159204D4F44450003404C464D4816
:1015F00040454A230102030A222121217D7D7D7D70
:101600007D7D7D7D7D7D7D7D7D7D7D797673716E3A
:101610006C6967656361605E5C5B595857555453EC
:1016200051504F4E4D4C4B4A494847464544434222
:101630004241403F3F3E3D3C3C3B3A3939383737E9
:101640003636353434333332313130302F2F2E2D7E
:101650002D2C2C2B2B2A2A292928282727262625FA
:10166000252524242323222221212020201F1F1E60
:101670001E1D1D1D1C1C1B1B1A1A1A1919181818BF
:101680001717161616151514141413131212121117
:10169000111010100F0F0E0E0E0D0D0C0C0C0B0B6D
:1016A0000A0A0909090808070707060605050404C8
:1016B0000403030202010101000000000000000019
:1016C000000000000000000000000000000000001A
:1016D000000000000000000000000000000000000A
:1016E00000000000000000000000000000000000FA
:1016F00000000000000000000000000000000001E9
:1017000001010200020001010101020001010101C9
:1017100002000200010101010101020002000200B9
:1017200002000200020001010101010102000101A9
:10173000020002000000000101010101000001019E
:10174000010101000101010101010000010100008E
:101750000000000001000000010102000101000082
:1017600001010101020002000101682FA901812F7E
:101770000023B9F40FE003BF00E002BF09E01DE35E
:101780000E940A4B10E0003021E0120710F000E048
:1017900009C001BF082F00FB07B701F907BF01E02F
:1017A00001C000E0862F089500E00093610002B9B7
:1017B00001BB04BB07BB0ABB00E0009365000093BC
:1017C000620003B902BB05BB08BB00B50B7F00BDBF
:1017D00000B50B7F00BD00E00093610002B901BBC2
:1017E00004BB07BB0ABB00E00093650000936200E6
:1017F00003B902BB05BB08BBBD9AC59A909A1C9A57
:101800001D9A1E9A1F9A04B30F6704BB02B10C60A5
:1018100002B9AC9AAB9AAA9AA99AA89AAE9AAD9A2A
:10182000AC9AAB9AAA9AA99AA89A1A981B9A01B349
:10183000006701BB9798949A959A9698AC9AAB9A40
:10184000AA9AA99AA89A0895002391F400E0009317
:10185000900019B902E00BB908E10AB920FB0EF4B7
:10186000579A06E0009395000FEF0CB95E9A089521
:101870000130E9F400E0009398001093990002E031
:1018800000939B0008E100939A0020FB2EF4009146
:101890009A00006800939A0006E000939D000FEF05
:1018A00000939C0000919B00006400939B000895AE
:1018B000592F482F80E090E008C02FE93FE02150E9
:1018C0003040E9F700C00000019680179107A8F3A7
:1018D000842F952F08959A938A9380E090E042D2C6
:1018E0000A3318F00753102F02C00053102F012F96
:1018F00010E0102F00E0110F110F110F110F802BAE
:10190000912B30D20A3318F00753102F02C0005326
:10191000102F012F302F20E0822B932B23D20A335C
:1019200018F00753102F02C00053102F012F10E0A2
:1019300044E00E94FE4A802B912B14D20A3318F007
:101940000753102F02C00053102F012F10E0802BDF
:10195000912B8C018991999108950E94A24B602E40
:101960002901B12F82E0A0E001E00093D80CAA2465
:101970009699A394BB249599B394969A959825C06B
:10198000949801E010E094DF00E00093EE0C0093E7
:10199000ED0C949A05E010E08BDF01E2B2D001E398
:1019A00011E086DF08E0ADD00091ED0C1091EE0C57
:1019B000011751F00091ED0C1091EE0C011721F080
:1019C000D1D10132B9F7A1E08A95813010F0AA2374
:1019D000B9F2AA2309F45FC000E00093EE0C009373
:1019E000ED0C8824992480E090E0772409E689D0E2
:1019F00008E087D0B7D10A33E9F7B4D10A33E9F761
:101A00006ADF4801AFD10A33E9F765DFC8018F3FCC
:101A10000FEF900751F0A6D10A33E9F7A3D10935AA
:101A200019F47724739401C07724E4EDFCE08082FC
:101A30009182E6EDFCE08083918360FABEF404E1DC
:101A400010E036DF04E45DD008E05BD08BD10A33D0
:101A5000E9F705E010E02CDF82015AD108E051D00F
:101A600008E04FD008E04DD008E04BD061FA4EF4CA
:101A700004E110E01DDFB71521F007E542D008E0D2
:101A800040D004E110E014DF05E43BD008E039D099
:101A900005E010E00DDF00E00093EE0C0093ED0C8C
:101AA0000A2D00FD969A00FF96980B2D00FD959A41
:101AB00000FF959800E00093D80C0A2FECE00C94FE
:101AC000B14B5E9A1B981A9A18D05E9BFECF1A985B
:101AD0001B9A08958A93802F082F02950F70005D3E
:101AE0000A3308F0095F0DD08F70805D082F0A332C
:101AF00008F0095F06D0899108955D9BFECF0CB96F
:101B00000895A99810919B00212F25FFFBCF0093EA
:101B10009C0008959A938A93802F082F44E60E9490
:101B2000E04A902F092F005DECDF04E6909F8019BA
:101B3000082F4AE00E94E04A902F092F005DE1DF64
:101B40000AE0909F8019805D082FDBDF89919991D1
:101B500008950E94A04B48015901DD24BB2052F496
:101B60009094A094B094000B8194900AA00AB00ABB
:101B70000DE2C7DF80E09AECAAE9BBE3CC241AC0EF
:101B8000DD2019F08201005DBCDF82019301AC0110
:101B9000BD010E942F4B801A910AA20AB30A8C0140
:101BA0009D014AE050E060E070E00E94794BC8017E
:101BB000D901C39409E0C016A8F484019501AC01D1
:101BC000BD010E94794B402E552466247724042DB4
:101BD000052906290729A1F28201005D92DFDD2493
:101BE000D394D3CF84019501AC01BD010E94794B00
:101BF000402E552466247724042D005D82DFEEE01C
:101C00000C94AF4B0E94A64B38015524A0E1B7E2DB
:101C100044240FC000E375DF8C01AD010E94EE4A41
:101C2000601A710A8D014AE050E00E940A4BD80107
:101C3000439405E04016D0F48301AD010E940A4BA5
:101C4000C801082F092B31F0082F005D5ADF5524F9
:101C50005394E2CF552021F0082F005D52DFDCCFF6
:101C600004E04016B8F600E24CDFD6CFE8E00C9472
:101C7000B54B10915209112311F02CDF089523E088
:101C800010E00AD0089520915209222311F040D08B
:101C9000089524E001D008950E94A44B3801822EBB
:101CA0005524A0E1B7E244240FC000E32ADF8C01F1
:101CB000AD010E94EE4A601A710A8D014AE050E0BF
:101CC0000E940A4BD801439405E04016F0F48301CA
:101CD000AD010E940A4BC80104E010E0242D30E061
:101CE000021B130B9924081519050CF7082F092B53
:101CF00031F0082F005D05DF55245394D8CF5520CF
:101D0000A1F2082F005DFDDED2CFEAE00C94B34BC8
:101D10009A938A93C8018C01012F10E0DBDE082F13
:101D2000D9DE8991999108950E94AA4BC801D901E1
:101D30008C019D01022F132F330F220B330BE8DF91
:101D40008C01E6DFE4E00C94B94BBA93AA93D80176
:101D500003C00C91D6DE11960C910023D1F7A99106
:101D6000B99108950091EE0C1091ED0C0117D1F38B
:101D70000091EE0C102F13951093EE0C10E00F70E5
:101D80001070F801E151F34F008108958A93802F7C
:101D9000082FC0DE08E2B5DE00E3B3DE08E5B1DE01
:101DA000082F98DE09E2ADDE899108950E94A34BC9
:101DB000EF97EF97EF972797A898992401E0009362
:101DC000590901E00093580905C004E110E070DDF5
:101DD00008E001BD992011F00C943F170EE915E0C1
:101DE000B4DF00914B09D2DF07EA15E0AEDF20E057
:101DF0008E0108571F4F0E94F01E00E00883AE01BD
:101E000048575F4F9E01205F3F4F8E010E94441D47
:101E1000802E00915609009357098820D9F20FE1CE
:101E2000801610F00EE1802E28E436E08E010E942C
:101E3000221D002351F626E436E08E010E94221D69
:101E4000002309F450C007EB10E00E94EB4880E04B
:101E50001CC0FE017096082F10E0000F111F000F2C
:101E6000111FE00FF11F008111812281338190E069
:101E7000FC01E254F74F008390E0FC01E254F74F7D
:101E80000081F7DE00E23DDE839590E0E82DF0E092
:101E900031978E179F07ECF21B981A9A80E008C0C2
:101EA00090E0FC01E254F74F008127DE5E9A8395B3
:101EB00090E0E82DF0E031978E179F078CF35E9B42
:101EC000FECF1A981B9A0FEF0E94974600935A096B
:101ED00009EC10E00E94EB4820915A090AE018E052
:101EE0000E94A44777CF21E436E08E010E94221D94
:101EF000002371F42EE336E08E010E94221D0023A0
:101F000039F42CE935E08E010E94221D002369F18D
:101F100000914B09083CB1F40CE810E00E94EB483A
:101F2000088919892A893B8931DF0AE3EADD0889B2
:101F300019892A893B89102F00914B090E94413A47
:101F4000A2DE48CF088919892A893B89009388072E
:101F50000C891D892E893F890093890722E012E0B0
:101F600000914B090E94CE4735CF27E935E08E011D
:101F70000E94221D0023A9F014E300914B090E9446
:101F8000874AC801282F14E100914B090E94BC1C0C
:101F9000892F90E0282F15E100914B090E94BC1C6D
:101FA00019CF23E935E08E010E94221D002341F064
:101FB00001E0009352090DEB15E10E94EB480ACFB6
:101FC0002FE835E08E010E94221D002341F000E041
:101FD0000093520902ED15E10E94EB48FBCE2AE87E
:101FE00035E08E010E94221D0023A9F014E3009128
:101FF0004B090E94874AC801282F16E100914B091E
:102000000E94BC1C892F90E0282F17E100914B09FA
:102010000E94BC1CDFCE26E835E08E010E94221D06
:10202000002339F42EE735E08E010E94221D0023A3
:10203000F9F080E014C0FE017096082F10E0000F48
:10204000111F000F111FE00FF11F0081118122816C
:10205000338190E0FC01E857F84F008383958815A1
:1020600050F38A94282D13E80EEF0E94CE47B2CE8B
:1020700028E735E08E010E94221D002371F425E738
:1020800035E08E010E94221D002339F423E735E05C
:102090008E010E94221D0023A1F100914B09083CF2
:1020A00081F40C891D892E893F89980148895989B5
:1020B0006A897B898A01102F00914B090E946F3930
:1020C00089CE80E014C0FE017096082F10E0000F4A
:1020D000111F000F111FE00FF11F008111812281DC
:1020E000338190E0FC01E857F84F00838395881511
:1020F00050F38A94282D13E000914B090E94CE479B
:1021000069CE2CE635E08E010E94221D002301F1EC
:1021100080E014C0FE017096082F10E0000F111F20
:10212000000F111FE00FF11F008111812281338107
:1021300090E0FC01E857F84F00838395881550F331
:102140008A94282D14E000914B090E94CE4742CE7C
:1021500025E635E08E010E94221D002339F421E698
:1021600035E08E010E94221D0023F9F080E014C0AA
:10217000FE017096082F10E0000F111F000F111FB5
:10218000E00FF11F008111812281338190E0FC0179
:10219000E857F84F00838395881550F38A94282DCB
:1021A00015E00EEF0E94CE4715CE2AE535E08E01F0
:1021B0000E94221D002381F00C891D892E893F89F0
:1021C000202F488959896A897B898A01102F0091BB
:1021D0004B090E94BC1CFECD24E535E08E010E9417
:1021E000221D002321F104EF10E00E94EB48BADD2C
:1021F000093719F0093509F0EDCD01E0801619F421
:1022000000914B0904C0088919892A893B8920E07B
:1022100016E00E94CE47002309F4DCCD01E00093D4
:102220004B0921E030E0A9010E94DC4AD3CD2DE426
:1022300035E08E010E94221D0023A1F001E08016EE
:1022400039F420E017E000914B090E94CE47C2CD3F
:1022500020E017E0488959896A897B89042F0E9408
:10226000CE47B8CD2AE435E08E010E94221D00231E
:1022700039F428E435E08E010E94221D0023D9F1B3
:1022800002E0801619F003E0801681F50EE100935C
:102290008807088919892A893B8900938907088951
:1022A00019892A893B89012F10E000938A0703E0EE
:1022B0008016A9F40C891D892E893F8900938B070C
:1022C0000C891D892E893F89012F10E000938C070E
:1022D00025E013E000914B090E94CE477BCD23E01F
:1022E00013E000914B090E94CE4774CD0BE011E042
:1022F0000E94EB486FCD23E435E08E010E94221D41
:10230000002379F001E0801619F400914B0904C014
:10231000088919892A893B8920E011E00E94CE476B
:1023200059CD20E435E08E010E94221D002349F1A1
:1023300003E000938807088919892A893B8900935B
:10234000890706E311E00E94EB480091890791DCC0
:102350000CE511E00E94EB4805DD093519F009375D
:1023600009F038CD22E013E00EEF0E94CE47009135
:10237000890700934B0921E030E0A9010E94DC4A63
:1023800029CD2DEF35E08E010E94221D002339F466
:102390002BEF35E08E010E94221D0023E1F0009119
:1023A0004B09083C11F4BED515CD00E00093880719
:1023B0000AE30093890722E012E000914B090E9492
:1023C000CE47002309F406CD00914B090E3F09F4D6
:1023D00001CDA8D5FFCC24EF35E08E010E94221D4F
:1023E000002309F43FC103E0801651F4488859885E
:1023F0006A887B880C891D892E893F89A02E0DC093
:1024000002E0801631F4488859886A887B88A42CB9
:1024100004C00EE81DE00E94EB4802E0801621F0A7
:1024200003E0801609F0D6CC00E000935809009331
:10243000590909B1023289F421E014E00EEF0E943B
:102440009D4A0AE010E034DA01E009B900934A0934
:1024500020E030E0A9010E94DC4A22E214E00EEF05
:102460000E949D4A0AE010E023DA02E209B90093D3
:102470004A0920E030E0A9010E94DC4A00E00E9405
:10248000064905C001E711E00E94EB484394A414FB
:1024900008F4DAC05524F201E55AF64F0081002312
:1024A000A9F30FEA1DE00E94EB48042DE2DB90E067
:1024B000992399F491E080E08F31D0F7082F0E94A2
:1024C000F41C002341F020E011E0082F0E94CE47C9
:1024D000002309F490E08395EFCF06EB1DE00E9406
:1024E000EB4880E00FC0841561F090E0FC01E55AF4
:1024F000F64F0081002329F025E01DE2082F0E94FD
:10250000BC1C83958F3178F300EC1DE00E94EB48F2
:102510002FEF1AEF042D0E94BC1C2EEF1DE2042D9C
:102520000E94BC1C002309F4ADCF04E610E0C0D922
:102530000DE0C7DA00E00E94761C0CE4C2DA00E08D
:102540000E94761C1B981A9A80E090ECA0E0B0E004
:1025500055246624772412C0FC013A2F3BBF069015
:1025600000E00BBF8F5F9F4FAF4FBF4F500C002D50
:10257000C4DA5E9A01E0600E00E0701E0FEF601694
:1025800007E1700648F3052DB8DA5E9A5E9BFECF30
:102590001A981B9A00E00E94761C06E592DA00E089
:1025A0000E94761C00E001C00395043638F410E068
:1025B000F801E65FF74F10811D32B1F70395202F28
:1025C00001C00395043638F410E0F801E65FF74FD8
:1025D00010811D32B1F7039510E001C0139518303A
:1025E00090F4602F062F0395422F242F239570E03F
:1025F000FB01E65FF74F308150E0FA01E65FF74FED
:102600004081341759F31830D1F40BEC1DE00E94CF
:10261000EB4801E456DA00E00E94761C07E451DA48
:1026200000E00E94761C20E017E0042D0E94CE47B7
:102630000CE211E03DD900E00093580927CF05EDE9
:102640001DE00E94EB4822CF0E94B44809B10093DC
:102650004A0920E030E0A9010E94DC4A01E0009331
:102660005909B8CB2FEE35E08E010E94221D0023C0
:1026700009F440C0B091580900E000935909009353
:10268000580980E001E0801611F4AEEF05C008891A
:1026900019892A893B89A02F0CE810E00E94EB4899
:1026A00090E005C00DE22DDA0DE52BDA93959A172F
:1026B00088F40BE526DA092FDCDA0AE322DA20E0D7
:1026C00011E0092F0E94CE47002361F30FE419DACD
:1026D0008395EACF0CE810E00E94EB48082F56DB08
:1026E00008E512E00E94EB48B093580901E000931E
:1026F000590970CB2BEE35E08E010E94221D00237C
:1027000009F459C001E0801619F4A0914B0905C0E5
:10271000088919892A893B89A02F00E0009359096B
:102720000093580903EA11E00E94EB4880E007E4B7
:1027300012E00E94EB480A2F9CDA0091EE0C1091F7
:10274000ED0C011791F00EDB802F823411F08236F0
:1027500009F4AA958E3411F08E3609F4A3950BE690
:1027600012E00E94EB480A2F84DA09E100938807FF
:1027700001E00093890722E013E00A2F0E94CE4770
:1027800004E610E095D809E10093880700E0009383
:10279000890722E013E00A2F0E94CE4704E610E0EA
:1027A00087D8813521F0813711F08B3131F601E086
:1027B000009359090FCB24EE35E08E010E94221DB3
:1027C000002309F48EC000E0009359090AE099D96A
:1027D00080E001C083958E3F08F078C089B920E081
:1027E00011E00EEF0E94CE470DE08BD980FB1EF466
:1027F0000BE287D902C00AE284D900915A0900236A
:1028000009F45DC0A0E056C0B0E0FD01E65FF74FFF
:1028100000810F3F09F04DC00A2F10E00F5F1F4FDE
:10282000F801E65FF74F00810F3F09F042C00A2F21
:1028300010E00D5F1F4FF801E65FF74F0081023097
:10284000C1F50A2F10E00E5F1F4FF801E65FF74F4A
:10285000408150E00A2F10E00D5F1F4FF801E65F46
:10286000F74F208130E0240F351F0A2F10E00B5F57
:102870001F4FF801E65FF74F008110E0020F131FB2
:102880000F3F20E01207A9F40CE712E00E94EB488A
:10289000082FEFD90FE812E00E94EB480A2F10E052
:1028A0000E5F1F4FF801E65FF74F0081E2D90AE0A3
:1028B00028D9A39500915A09A01708F4A5CF009133
:1028C000EE0C1091ED0C011709F484CF00914A0928
:1028D00009B901E0009359090DE013D900E211D9BB
:1028E00079CA2FED35E08E010E94221D002391F15F
:1028F00004E000938807088919892A893B89009395
:10290000890722E013E00EEF0E94CE4705E912E0AE
:102910000E94EB4800E814E82EE130E0488959892C
:102920006A897B894F5F5F4F6F4F7F4F0E94534B88
:1029300010D900EB12E00E94EB48088919892A8916
:102940003B8909B900934A0920E030E0A9010E94BF
:10295000DC4A40CA27ED35E08E010E94221D00238B
:1029600009F442C001E0801631F400E1402E552404
:102970006624772404C0488859886A887B8800ECDC
:1029800011E00E94EB482BC00091570910915609A5
:102990000117A1F080E090E0A0E0B0E0AA2400914F
:1029A000570910E0F801E857F94F0081E7E5F9E031
:1029B0001081139510835DD900E2A3D88F5F9F4FDC
:1029C000AF4FBF4F84159505A605B705E8F2AA20BD
:1029D00031F40DE096D80AE094D8AA24A39480E0BC
:1029E00090E0A0E0B0E0EECF22ED35E08E010E9455
:1029F000221D002309F461C0088919892A893B89AD
:102A0000A02F4C885D886E887F8804EB12E00E94BE
:102A1000EB480A2F2ED90FEB12E00E94EB488201FF
:102A200032D909EC12E00E94EB4880E00CC008E1CA
:102A30000093880701E00093890722E013E0082F44
:102A40000E94CE478395A81790F70AED12E00E94E6
:102A5000EB4814C00EE1009388070FEF009389073D
:102A600003E000938A0723E013E0082F0E94CE477B
:102A70008395A81778F782010E94580C0091EE0CFC
:102A80001091ED0C011709F0A5C980E00FC00EE10F
:102A90000093880700E00093890700E000938A070D
:102AA00023E013E0082F0E94CE478395A81778F7FC
:102AB00082010E94580C80E0DCCF2EEC35E08E01C4
:102AC000C1D7002309F431C100E0009359090091F6
:102AD0004B090093880721E015E00EEF0E94CE47D6
:102AE00001E0801641F520E130E0A9010E94D04AC2
:102AF000802E80E090E0E82DF0E031978E179F0760
:102B00000CF042C0E82FF0E07196AF010E94D04A6D
:102B100010E020E030E0FE017096482F50E0440FB6
:102B2000551F440F551FE40FF51F008311832283A7
:102B300033838395DFCF05E1801610F004E1802E0A
:102B400020E130E0082DA9010E94DC4A80E015C098
:102B5000FE017096082F10E0000F111F000F111FCB
:102B6000E00FF11F0081118122813381E82FF0E015
:102B70007196AF010E94DC4A839590E0E82DF0E069
:102B800031978E179F0724F30CE810E00E94EB4862
:102B90000BE50E94810D80E004C00DE50E94810DCF
:102BA000839590E0E82DF0E031978E179F07D4F4DD
:102BB000FE017096082F10E0000F111F000F111F6B
:102BC000E00FF11F008111812281338152D890E002
:102BD000E82DF0E032978E179F07FCF60DE20E9479
:102BE000810DDECF0091EE0C1091ED0C011709F074
:102BF00098C00CE810E00E94EB4880E018C0FE018D
:102C00007096082F10E0000F111F000F111FE00F2A
:102C1000F11F0081118122813381102F00914B0916
:102C20000E94784A26D800E20E94810D839590E0A8
:102C3000E82DF0E031978E179F07A4F6FE017096FD
:102C4000082F10E0000F111F000F111FE00FF11FE0
:102C50000081118122813381083CF9F000914B09F8
:102C6000043688F100914B090E3668F504E317E14C
:102C7000FE017096282F30E0220F331F220F331FE2
:102C8000E20FF31F408151816281738150E0040F94
:102C9000151FF80104910230B1F4FE017096082F5F
:102CA00010E0000F111F000F111FE00FF11F008136
:102CB000118122813381102F00914B090E94413AEA
:102CC0000E94430EB0CF0CEF16E1FE017096282F44
:102CD00030E0220F331F220F331FE20FF31F40811A
:102CE00051816281738150E0040F151FF801049136
:102CF000023009F084CFFE017096082F10E0000F1B
:102D0000111F000F111FE00FF11F0081118122819F
:102D10003381102F00914B090E94874A0E94430E75
:102D200082CF01E00093590955C829EC35E08E01A6
:102D300089D6002309F447C0488859886A887B8867
:102D40008C899D89AE89BF8900E000935909A0E074
:102D50004A1608F108E10093880701E0009389070B
:102D600022E013E00A2F0E94CE47A395F1CF0EE197
:102D7000009388070FEF0093890703E000938A0709
:102D800023E013E00A2F0E94CE47A3954A1678F756
:102D90008C010E94580CA0E00FC00EE10093880740
:102DA00000E00093890700E000938A0723E013E026
:102DB0000A2F0E94CE47A3954A1678F78C010E94ED
:102DC000580CA0E0E3CF25EC35E08E013BD6002384
:102DD00069F0088919892A893B8900934B0921E008
:102DE00030E0A9010E94DC4A0C94EA0E20EC35E0A8
:102DF0008E0128D6002331F42EEB35E08E0122D649
:102E0000002321F00E9465460C94EA0E29EB35E080
:102E10008E0118D6002319F03CD00C94EA0E25EB55
:102E200035E08E010FD6002381F002E0801640F0DD
:102E3000088919892A893B890E94BC3E0C94EA0EB4
:102E400001E00E94BC3E0C94EA0E2EEA35E08E01B1
:102E5000F9D5002331F42AEA35E08E01F3D50023B9
:102E600021F0992493940C94EA0E0CE810E00E944F
:102E7000EB4808EE1DE00E94EB480C94EA0E00E0DF
:102E800000935909EF96EF96EF962796EBE00C9496
:102E9000B24B03E319E00E94EB4805E519E00E94FC
:102EA000EB480BE719E00E94EB4800EA19E00E94AA
:102EB000EB4809EE19E00E94EB4800E31AE00E949B
:102EC000EB4807E61AE00E94EB480DE81AE00E9482
:102ED000EB4808EC1AE00E94EB4806E01BE00E9479
:102EE000EB4802E21BE00E94EB480CE41BE00E946E
:102EF000EB4807E81BE00E94EB480CEC1BE00E944B
:102F0000EB4805E11CE00E94EB4809E51CE00E944B
:102F1000EB4806E91CE00E94EB4803EE1CE00E942F
:102F2000EB4808950E94AA4B00914B09083C09F018
:102F3000B9C088E10CEF1DE00E94EB48082F0E9409
:102F4000C60E0AE30E94810D182F00914B090E94C2
:102F5000413A0E94430E839509E11EE00E94EB482E
:102F6000082F0E94C60E0AE30E94810D182F0091BF
:102F70004B090E94413A0E94430E839506E31EE0EE
:102F80000E94EB48082F0E94C60E0AE30E94810DA2
:102F9000182F00914B090E94413A0E94430E8395DD
:102FA000839503E51EE00E94EB48082F0E94C60EA1
:102FB0000AE30E94810D182F00914B090E94413AAB
:102FC0000E94430E8395839500E71EE00E94EB4824
:102FD000082F0E94C60E0AE30E94810D182F00914F
:102FE0004B090E94413A0E94430E83950DE81EE072
:102FF0000E94EB48082F0E94C60E0AE30E94810D32
:10300000182F00914B090E94413A0E94430E83956C
:103010000AEA1EE00E94EB48082F0E94C60E0AE34F
:103020000E94810D182F00914B090E94413A0E9485
:10303000430E839507EC1EE00E94EB48082F0E9488
:10304000C60E0AE30E94810D182F00914B090E94C1
:10305000413A0E94430E839504EE1EE00E94EB4825
:10306000082F0E94C60E0AE30E94810D182F0091BE
:103070004B090E94413A0E94430E8395839501E0DB
:103080001FE00E94EB48082F0E94C60E0AE30E9430
:10309000810D182F00914B090E94413A0E94430E66
:1030A000839521C480E008E013E00E94EB48082FDC
:1030B0000E94C60E0CEA1DE00E94EB48A82FB0E06B
:1030C0001596FD01E65FF74F00810E94C60E8395BD
:1030D00007E313E00E94EB48082F0E94C60E0CEA9B
:1030E0001DE00E94EB48A82FB0E01596FD01E65FB9
:1030F000F74F00810E94C60E839506E513E00E94FB
:10310000EB48082F0E94C60E0CEA1DE00E94EB4817
:10311000A82FB0E01596FD01E65FF74F00810E94F1
:10312000C60E839505E713E00E94EB48082F0E9426
:10313000C60E0CEA1DE00E94EB48A82FB0E01596E1
:10314000FD01E65FF74F00810E94C60E839504E9FA
:1031500013E00E94EB48082F0E94C60E0CEA1DE007
:103160000E94EB48A82FB0E01596FD01E65FF74FEF
:1031700000810E94C60E839503EB13E00E94EB488A
:10318000082F0E94C60E0CEA1DE00E94EB48A82FF3
:10319000B0E01596FD01E65FF74F00810E94C60E74
:1031A000839502ED13E00E94EB48082F0E94C60EA3
:1031B0000CEA1DE00E94EB48A82FB0E01596FD0137
:1031C000E65FF74F00810E94C60E839501EF13E082
:1031D0000E94EB48082F0E94C60E0CEA1DE00E94D8
:1031E000EB48A82FB0E01596FD01E65FF74F008190
:1031F0000E94C60E839500E114E00E94EB48082F60
:103200000E94C60E0CEA1DE00E94EB48A82FB0E019
:103210001596FD01E65FF74F00810E94C60E83956B
:103220000FE214E00E94EB48082F0E94C60E0CEA41
:103230001DE00E94EB48A82FB0E01596FD01E65F67
:10324000F74F00810E94C60E83950EE414E00E94A1
:10325000EB48082F0E94C60E0CEA1DE00E94EB48C6
:10326000A82FB0E01596FD01E65FF74F00810E94A0
:10327000C60E83950DE614E00E94EB48082F0E94CD
:10328000C60E0CEA1DE00E94EB48A82FB0E0159690
:10329000FD01E65FF74F00810E94C60E83950CE8A2
:1032A00014E00E94EB48082F0E94C60E0CEA1DE0B5
:1032B0000E94EB48A82FB0E01596FD01E65FF74F9E
:1032C00000810E94C60E83950BEA14E00E94EB4831
:1032D000082F0E94C60E0CEA1DE00E94EB48A82FA2
:1032E000B0E01596FD01E65FF74F00810E94C60E23
:1032F00083950AEC14E00E94EB48082F0E94C60E4A
:103300000CEA1DE00E94EB48A82FB0E01596FD01E5
:10331000E65FF74F00810E94C60E839509EE14E028
:103320000E94EB48082F0E94C60E0CEA1DE00E9486
:10333000EB48A82FB0E01596FD01E65FF74F00813E
:103340000E94C60E839508E015E00E94EB48082F06
:103350000E94C60E0CEA1DE00E94EB48A82FB0E0C8
:103360001596FD01E65FF74F00810E94C60E83951A
:1033700007E215E00E94EB48082F0E94C60E0CEAF7
:103380001DE00E94EB48A82FB0E01596FD01E65F16
:10339000F74F00810E94C60E839506E415E00E9457
:1033A000EB48082F0E94C60E0CEA1DE00E94EB4875
:1033B000A82FB0E01596FD01E65FF74F00810E944F
:1033C000C60E839505E615E00E94EB48082F0E9483
:1033D000C60E0CEA1DE00E94EB48A82FB0E015963F
:1033E000FD01E65FF74F00810E94C60E839504E859
:1033F00015E00E94EB48082F0E94C60E0CEA1DE063
:103400000E94EB48A82FB0E01596FD01E65FF74F4C
:1034100000810E94C60E839503EA15E00E94EB48E6
:10342000082F0E94C60E0CEA1DE00E94EB48A82F50
:10343000B0E01596FD01E65FF74F00810E94C60ED1
:10344000839502EC15E00E94EB48082F0E94C60EFF
:103450000CEA1DE00E94EB48A82FB0E01596FD0194
:10346000E65FF74F00810E94C60E839501EE15E0DE
:103470000E94EB48082F0E94C60E0CEA1DE00E9435
:10348000EB48A82FB0E01596FD01E65FF74F0081ED
:103490000E94C60E83950EEE12E00E94EB480E9439
:1034A000B20E00E016E00E94EB48082F0E94C60E04
:1034B0000CEA1DE00E94EB48A82FB0E01596FD0134
:1034C000E65FF74F00810E94C60E83950CE216E07E
:1034D0000E94EB48082F0E94C60E0CEA1DE00E94D5
:1034E000EB48A82FB0E01596FD01E65FF74F00818D
:1034F0000E94C60E83950BE416E00E94EB48082F4D
:103500000E94C60E0CEA1DE00E94EB48A82FB0E016
:103510001596FD01E65FF74F00810E94C60E839568
:103520000AE616E00E94EB48082F0E94C60E0CEA3D
:103530001DE00E94EB48A82FB0E01596FD01E65F64
:10354000F74F00810E94C60E839509E816E00E949D
:10355000EB48082F0E94C60E0CEA1DE00E94EB48C3
:10356000A82FB0E01596FD01E65FF74F00810E949D
:10357000C60E839508EA16E00E94EB48082F0E94C9
:10358000C60E0CEA1DE00E94EB48A82FB0E015968D
:10359000FD01E65FF74F00810E94C60E839507ECA0
:1035A00016E00E94EB48082F0E94C60E0CEA1DE0B0
:1035B0000E94EB48A82FB0E01596FD01E65FF74F9B
:1035C00000810E94C60E839506EE16E00E94EB482D
:1035D000082F0E94C60E0CEA1DE00E94EB48A82F9F
:1035E000B0E01596FD01E65FF74F00810E94C60E20
:1035F000839505E017E00E94EB48082F0E94C60E55
:103600000CEA1DE00E94EB48A82FB0E01596FD01E2
:10361000E65FF74F00810E94C60E839504E217E033
:103620000E94EB48082F0E94C60E0CEA1DE00E9483
:10363000EB48A82FB0E01596FD01E65FF74F00813B
:103640000E94C60E839503E417E00E94EB48082F02
:103650000E94C60E0CEA1DE00E94EB48A82FB0E0C5
:103660001596FD01E65FF74F00810E94C60E839517
:1036700002E617E00E94EB48082F0E94C60E0CEAF3
:103680001DE00E94EB48A82FB0E01596FD01E65F13
:10369000F74F00810E94C60E839501E817E00E9453
:1036A000EB48082F0E94C60E0CEA1DE00E94EB4872
:1036B000A82FB0E01596FD01E65FF74F00810E944C
:1036C000C60E839500EA17E00E94EB48082F0E947F
:1036D000C60E0CEA1DE00E94EB48A82FB0E015963C
:1036E000FD01E65FF74F00810E94C60E83950FEB48
:1036F00017E00E94EB48082F0E94C60E0CEA1DE05E
:103700000E94EB48A82FB0E01596FD01E65FF74F49
:1037100000810E94C60E83950EED17E00E94EB48D3
:10372000082F0E94C60E0CEA1DE00E94EB48A82F4D
:10373000B0E01596FD01E65FF74F00810E94C60ECE
:1037400083950DEF17E00E94EB48082F0E94C60EEC
:103750000CEA1DE00E94EB48A82FB0E01596FD0191
:10376000E65FF74F00810E94C60E83950CE118E0DA
:103770000E94EB48082F0E94C60E0CEA1DE00E9432
:10378000EB48A82FB0E01596FD01E65FF74F0081EA
:103790000E94C60E83950BE318E00E94EB48082FA9
:1037A0000E94C60E0CEA1DE00E94EB48A82FB0E074
:1037B0001596FD01E65FF74F00810E94C60E8395C6
:1037C0000AE518E00E94EB48082F0E94C60E0CEA9A
:1037D0001DE00E94EB48A82FB0E01596FD01E65FC2
:1037E000F74F00810E94C60E839509E718E00E94FA
:1037F000EB48082F0E94C60E0CEA1DE00E94EB4821
:10380000A82FB0E01596FD01E65FF74F00810E94FA
:10381000C60E839508E918E00E94EB48082F0E9425
:10382000C60E0CEA1DE00E94EB48A82FB0E01596EA
:10383000FD01E65FF74F00810E94C60E839507EBFE
:1038400018E00E94EB48082F0E94C60E0CEA1DE00B
:103850000E94EB48A82FB0E01596FD01E65FF74FF8
:1038600000810E94C60E839506ED18E00E94EB4889
:10387000082F0E94C60E0CEA1DE00E94EB48A82FFC
:10388000B0E01596FD01E65FF74F00810E94C60E7D
:10389000839505EF18E00E94EB48082F0E94C60EA2
:1038A0000CEA1DE00E94EB48A82FB0E01596FD0140
:1038B000E65FF74F00810E94C60E839504E119E090
:1038C0000E94EB48082F0E94C60E0CEA1DE00E94E1
:1038D000EB48A82FB0E01596FD01E65FF74F008199
:1038E0000E94C60E8395E4E00C94B94B9A938A9398
:1038F000902F80E000915709109156090117D1F3DC
:1039000040E050E060E070E00091570910915609E6
:103910000117A1F48A019B01A801B9014F5F5F4F14
:103920006F4F7F4F013EE3E91E07E4E02E07E0E022
:103930003E0750F3082F89919991089500915709F6
:1039400010E0F801E857F94F0081E7E5F9E0108150
:1039500013951083282F30E0F901E65FF74F0083BD
:10396000992341F0082F10E0F801E65FF74F00813E
:103970000E94810D8395C4CF0E94AA4B902FA12F46
:10398000B22FA0938807B093890700EF00938A07AE
:1039900005E500938B070FE000938C070AEA00937C
:1039A0008D0726E01DE0092F0E945347802F0091CC
:1039B0005909002349F00CE810E00E94EB48282F39
:1039C0000EEB18E00E94A4470AE010E00E94580C99
:1039D0001A2F092F0E94784A0B1711F401E001C039
:1039E00000E0E4E00C94B94B0F3130F410E0F80142
:1039F000E55AF64F00810895043650F00E3640F433
:103A000010E004561040F801E558F64F0081089583
:103A100000E00895A80100E001C00395083C88F487
:103A200010E0F901E00FF11F608110E0FA01E00FF2
:103A3000F11F608310E0F901E00FF11F10811123E5
:103A400061F70895A80100E010E0FA01E00FF11F0E
:103A5000608110E0F901E00FF11F1081611791F40E
:103A6000039510E0FA01E00FF11F1081112339F4E2
:103A700010E0F901E00FF11F1081112321F0093C42
:103A800018F3089500E008950E94A74BD901CA01D8
:103A9000442401C043945524FC01E40DF51D20810C
:103AA0002032C1F32CE3421608F041C05524FC013A
:103AB000E40DF51D20812223D1F120E021C0552401
:103AC000FC01E40DF51D3081313670F05524FC0108
:103AD000E40DF51D30813B3738F45524FC01E40D2D
:103AE000F51D30813F7530835524FC01E40DF51D33
:103AF000408130E0F801E20FF31F408323954394A7
:103B00005524FC01E40DF51D3081303350F055246F
:103B1000FC01E40DF51D30813B3718F430E143160C
:103B200070F240E030E0F801E20FF31F4083E02F35
:103B3000F12F0081002311F400E0A6C066249EC08E
:103B400043945524FC01E40DF51D00810032C1F3BE
:103B50005524FC01E40DF51D0081002319F4639444
:103B6000062D92C000E010E020E030E0462D50E04D
:103B7000440F551F440F551FFD01E40FF51F00832F
:103B800011832283338342C0062D10E0000F111FE2
:103B9000000F111FFD01E00FF11F00811181228133
:103BA00033814AE050E060E070E00E942F4B462DE8
:103BB00050E0440F551F440F551FFD01E40FF51F42
:103BC00000831183228333835524FC01E40DF51D0A
:103BD000008110E000531040212F220F220B322FC2
:103BE000462D50E0440F551F440F551FFD01E40FB3
:103BF000F51F4081518162817381400F511F621F07
:103C0000731F408351836283738343940CE3401694
:103C1000A0F55524FC01E40DF51D0081002321F4DD
:103C200002E0600E062D30C05524FC01E40DF51DA8
:103C300000810B33E1F05524FC01E40DF51D0081FA
:103C40000A33A9F05524FC01E40DF51D00810C3266
:103C500071F05524FC01E40DF51D00810E3239F0A0
:103C60005524FC01E40DF51D0081003281F400E2D1
:103C70005524FC01E40DF51D008363940EE16016EC
:103C800008F45FCF6394062DE7E00C94B64B0091E7
:103C90005209002309F478CF5524FC01E40DF51DE9
:103CA0000081003308F446C05524FC01E40DF51DE5
:103CB00000810A33F8F5062D10E0000F111F000FE8
:103CC000111FFD01E00FF11F00811181228133815D
:103CD00044E00E944B4B462D50E0440F551F440FCB
:103CE000551FFD01E40FF51F0083118322833383E9
:103CF0005524FC01E40DF51D008110E00053104037
:103D0000212F220F220B322F462D50E0440F551F3A
:103D1000440F551FFD01E40FF51F40815181628161
:103D20007381400F511F621F731F40835183628351
:103D300073836BCF5524FC01E40DF51D0081013424
:103D400008F463CF5524FC01E40DF51D00810B3709
:103D500008F05BCF5524FC01E40DF51D00810F75C3
:103D60000083062D10E0000F111F000F111FFD0131
:103D7000E00FF11F008111812281338144E00E9414
:103D80004B4B462D50E0440F551F440F551FFD016E
:103D9000E40FF51F00831183228333835524FC0134
:103DA000E40DF51D008110E007531040212F220F74
:103DB000220B322F462D50E0440F551F440F551F44
:103DC000FD01E40FF51F4081518162817381400F35
:103DD000511F621F731F408351836283738315CF0A
:103DE0000E94AA4BC801A22FB1E016C008E00E94B1
:103DF000810D00E20E94810D08E00E94810D0A2FD2
:103E0000A02FAA95002391F72FEA3DE08C0102DE56
:103E1000A02F8C010E94A50EBB23A9F10E94B20E17
:103E2000102F1050C9F31A9551F3175099F01250F2
:103E300029F0135019F01E5079F319C000E0B0E0DA
:103E4000FC01EA0FFB1F00839C010FEA1DE0E2DD8D
:103E500001E01AC0A13000F3AA9508E00E94810D8C
:103E600000E20E94810D08E00E94810DD5CFAC33A5
:103E700098F62A2F30E0FC01E20FF31F00830E9426
:103E8000810DA395C9CF00E0E4E00C94B94B0E94EA
:103E9000AA4B902F812F983050F5883040F5092F8C
:103EA00010E00F5F1F4F40E450E00E94EE4AD8013F
:103EB000082F10E00F5F1F4F40E450E00E94EE4AD1
:103EC00020E011C0422F50E0400F511FFA01EA5389
:103ED000F64F3081422F50E04A0F5B1FFA01EA5340
:103EE000F64F30832395203468F3092F03D0E4E0A4
:103EF0000C94B94B9A938A93902F973011F490E0D9
:103F000001C0939580E007C0182F092F27D2182FE2
:103F1000092F2BD183958F31B8F31FE1092F1ED2C2
:103F20001FE1092FD3D0F801EA53F64F00810E9418
:103F3000390E10E2092F12D210E2092FC7D0F80172
:103F4000EA53F64F00810E94390E899199910895A4
:103F5000005049F00A9561F00A9579F00A9591F0C0
:103F60000A95A9F008950DEB14E10E94EB4808951D
:103F700001ED14E10E94EB4808950FED14E10E9459
:103F8000EB48089502EF14E10E94EB48089502E027
:103F900015E10E94EB4808959A938A93802F912F00
:103FA000E9EFF5E11491E0EFF5E104910E946A2E4A
:103FB00022E0082F10E00E944C0EEAEFF5E1149188
:103FC000E1EFF5E104910E946A2E22E0092F10E052
:103FD0000E944C0EEBEFF5E11491E2EFF5E1049154
:103FE0000E946A2E192F082F71D00E94430E8991CA
:103FF000999108958A93E3EFF5E11491EAEEF5E1E2
:1040000004910E946A2E80E004C000E20E94810DAB
:1040100083958634D0F3E3EFF5E11491EAEEF5E110
:1040200004910E946A2E899108959A938A9390919F
:10403000DA0980E00CC0182F0091EB0D03958ED1AA
:1040400008E00E94810D00E20E94810D83958F316E
:1040500090F380E00BC0182F092F03957FD108E063
:104060000E94810D0CE70E94810D83958F3198F39A
:104070009093EB0DE7EFF5E11491EEEEF5E104918D
:104080000E946A2E092F0E94390E899199910895F4
:10409000093031F4133020F0143110F401E00895A8
:1040A000083021F41F3110F401E00895083030F495
:1040B000103211F01F3111F401E00895083020F49E
:1040C000103210F402E0089500E00895682F202FC8
:1040D000812F222371F48F3138F4082F10E0000F64
:1040E000111F00501E4F39C0082F10E0015E1D4FF8
:1040F00034C08F3149F4022F10E040E450E00E94B8
:10410000EE4A025C1F4F29C0803249F4022F10E0B2
:1041100040E450E00E94EE4A015C1F4F1EC0283070
:1041200029F4082F10E0005E1F4F17C0293029F432
:10413000082F10E0055F1F4F10C0022F10E0015044
:10414000104040E450E00E94EE4A980102E0809F57
:104150008001020F131F005C1F4F003422E0120782
:1041600010F000E010E0862F08959A938A93902F24
:10417000812F8F3108F042C0182F092FA7DFF801D7
:10418000EA53F64F20813181203004E0300748F0B7
:10419000182F092F9BDFF801EA53F64F018107FF23
:1041A0000BC0182F092F92DFF801EA53F64F008158
:1041B00011810E94430E22C0182F092F87DFF801BA
:1041C000EA53F64F018105FF0DC00FE30E94810DF8
:1041D0000FE30E94810D0FE30E94810D0FE30E9407
:1041E000810D0CC00DE20E94810D0DE20E94810D37
:1041F0000DE20E94810D0DE20E94810D899199913D
:1042000008959A938A930091CA0C002351F000E01C
:104210009FDE0E94B20E093521F0093711F000E04F
:104220005CC0E8ECFCE00081118120E030E040E07F
:1042300052E060E070E00E942F4BA801B9014050AD
:1042400050426F4F7F4F10E080E090E017C00C01AC
:1042500022243324040E151E261E371EF001322D93
:104260003BBF069000E00BBFFC01EA53F64F008213
:10427000FC01EA53F64F0081100F0196803002E0F6
:10428000900728F300E015C0202F30E0F901E55A2F
:10429000F64F2081222361F440E050E422E0029FA7
:1042A000900120503E4FF901EA53F64F408351836D
:1042B00003950F3148F31F3F21F40091DA090830CC
:1042C00008F00ED000E00093CA0C0091DD09053023
:1042D00018F000E00093DD0901E0899199910895BB
:1042E0003B2F2A2FE0E0F0E006C000E0DF01AA53F8
:1042F000B64F0C933196E03200E0F007B0F3E0E205
:10430000F0E006C005E5DF01AA53B64F0C933196E5
:10431000E03400E0F007B0F3E0E4F0E009C000E0D2
:1043200010E4DF01AA53B64F0D931C9311973296F8
:10433000E03002E0F00798F300E00093DA0901E0D2
:104340000093D50900E20093DC0900E20093DE0946
:1043500000E00093D309A22FB32F08959A938A9374
:104360006297602F212FCE010896E8EFF7E930E041
:104370008C014AE050E00E948F4BCE01E2E0F8E968
:1043800030E08C0148E050E00E948F4B203211F069
:104390002F3151F42395122FFE0170E0E60FF71F25
:1043A00000810E946A2E10C02F3158F42395122FDD
:1043B000FE01389670E0E60FF71F00810E946A2E1A
:1043C00003C001E20E94810D62968991999108953E
:1043D0008A93802F03C000E20E94810D082F802F56
:1043E0008A950023C1F7899108950E94AB4B80E024
:1043F00005C00CE810E00E94EB4883958C33C8F3AD
:1044000011E001E00E946A2E0EE11FE00E94EB48DD
:1044100008E31FE00E94EB4807E2DADF03E51FE054
:104420000E94EB4800E61FE00E94EB4807E2D0DF65
:104430000BE71FE00E94EB4802E81FE00E94EB48F8
:1044400007E2C6DF0DE91FE00E94EB480BEA1FE020
:104450000E94EB4807E2BCDF06EC1FE00E94EB483D
:1044600004ED1FE00E94EB4807E2B2DF0FEE1FE011
:104470000E94EB480DEF1FE00E94EB4807E2A8DF27
:1044800008E110E10E94EB4806E210E10E94EB48CF
:1044900007E29EDF01E410E10E94EB480FE410E127
:1044A0000E94EB4807E294DF0AE610E10E94EB4825
:1044B00008E710E10E94EB4807E28ADF03E910E118
:1044C0000E94EB4801EA10E10E94EB4807E280DF1E
:1044D0000CEB10E10E94EB480AEC10E10E94EB4863
:1044E00007E276DF05EE10E10E94EB4803EF10E1F2
:1044F0000E94EB4807E26CDF0EE011E10E94EB48FE
:104500000CE111E10E94EB4807E262DF07E311E1F1
:104510000E94EB4805E411E10E94EB4807E258DFF6
:1045200000E611E10E94EB480EE611E10E94EB4823
:1045300007E24EDF09E811E10E94EB4807E911E1CB
:104540000E94EB4807E244DF02EB11E10E94EB48D6
:1045500000EC11E10E94EB4807E23ADF0BED11E1BC
:104560000E94EB4809EE11E10E94EB4807E230DFC0
:1045700004E012E10E94EB4802E112E10E94EB48E4
:1045800007E226DF0DE212E10E94EB480BE312E1A5
:104590000E94EB4806E512E10E94EB4801E712E1B8
:1045A0000E94EB480CE812E10E94EB4807EA12E196
:1045B0000E94EB4802EC12E10E94EB480DED12E183
:1045C0000E94EB4808EF12E10E94EB4803E113E17F
:1045D0000E94EB480EE213E10E94EB4809E413E16C
:1045E0000E94EB4804E613E10E94EB480FE713E159
:1045F0000E94EB48E8ECFCE000811181012B29F4DA
:104600000FE114E10E94EB4804C000ED13E10E94A9
:10461000EB480EE614E10E94EB4880E001C0839570
:104620008132F8F490E006C0A23019F4182F092F57
:104630009CDD9395933198F7182F092F29DDA02F32
:10464000AA23B9F3182F092F89DEA13069F7182F93
:10465000092F3CDDF801EA53F64F00810E94390E24
:10466000E8CFE3DCE4EFF5E11491EBEEF5E1049142
:104670000E946A2E06EC19E00E94A50EE5EFF5E116
:104680001491ECEEF5E104910E946A2EE8ECFCE056
:10469000008111810E94430EE6EFF5E11491EDEEE9
:1046A000F5E104910E946A2EE8ECFCE000811181A2
:1046B00020E030E040E052E060E070E00E942F4BEC
:1046C000005010422F4F3F4F0E94940EE3E00C9495
:1046D000BA4B0E94A14BEF97EA97DA95BE0164525C
:1046E0007F4FEAE0F8E930E08B0141E250E00E94C0
:1046F0008F4BA0E0BA2FBA2ECA2E24EF3FE0A901BB
:104700000E94D04A053511F40C94872D1A2F0B2FD7
:1047100043DC1A2F0B2F22DE9090DA090091520908
:10472000002319F000E1A02E02C00AE0A02E0E9492
:10473000B20E902F9B31D9F50E94B20E902F9B356F
:1047400019F40E94B20E902F943421F4BB2389F007
:10475000BA950FC0933411F4B3950BC0913421F482
:10476000AA2339F0AA9505C0923419F4A03208F4AE
:10477000A395FE01E452FF4F0A2F10E0E00FF11F56
:1047800000810B1738F4FE01E452FF4FB0E0EA0F4E
:10479000FB1FB081BC1521F4AB1511F40C94212E34
:1047A0001A2F0B2FF9DBCB2EBA2E0C94212E903220
:1047B00009F044C01A2F0B2F6BDC023011F00C945F
:1047C000212E80E090E21A2F0B2F80DCF801EA53B3
:1047D000F64F008111810827192700831183BB231D
:1047E00029F58A2F02E0809F800100501E4FF801BA
:1047F000EA53F64F018105FD16C090E0FC01E55A31
:10480000F64F0081002379F014E2082F0E943E2E1B
:1048100022E0829F20E0020E22E0121EF001EA5305
:10482000F64F008311830A2F0E9424381A2F0B2F72
:104830009CDC01E00093CA0C0C94212E9D3509F0FC
:104840004CC01A2F0B2F8ADD1A2F0B2F21DC0130C1
:10485000B9F41A2F0B2F3ADCF801EA53F64F008116
:10486000039500831A2F0B2F31DCF801EA53F64F22
:1048700000810E94390E01E00093CA0C0C94212E95
:10488000023011F00C94212E1A2F0B2F1FDCF8018F
:10489000EA53F64F008111810F7F13700F3F23E021
:1048A000120711F40C94212E1A2F0B2F0FDCF80194
:1048B000EA53F64F008111810F5F1F4F0083118370
:1048C0001A2F0B2F52DCBB2319F40A2F0E94243815
:1048D00001E00093CA0C0C94212E9B3509F04AC0CC
:1048E0001A2F0B2F3BDD1A2F0B2FD2DB0130B9F41F
:1048F0001A2F0B2FEBDBF801EA53F64F00810A95D4
:1049000000831A2F0B2FE2DBF801EA53F64F0081E8
:104910000E94390E01E00093CA0C0C94212E023043
:1049200011F00C94212E1A2F0B2FD0DBF801EA5333
:10493000F64F008111810F7F1370012B11F40C943D
:10494000212E1A2F0B2FC2DBF801EA53F64F0081FC
:10495000118101501040008311831A2F0B2F05DCA9
:10496000BB2319F40A2F0E94243801E00093CA0CDB
:104970000C94212E9D3709F050C01A2F0B2F88DB85
:104980000130B9F41A2F0B2FA1DBF801EA53F64FCF
:1049900000810A0D00831A2F0B2F98DBF801EA53D0
:1049A000F64F00810E94390E01E00093CA0C0C946E
:1049B000212E023011F00C94212E1A2F0B2F86DBA2
:1049C000F801EA53F64F008111810F7F13702FEF2A
:1049D00033E04A2D50E0241B350B0217130710F06B
:1049E0000C94212E8A2D90E01A2F0B2F6FDBF801EB
:1049F000EA53F64F00811181080F191F00831183BC
:104A00001A2F0B2FB2DBBB2319F40A2F0E94243874
:104A100001E00093CA0C0C94212E9B3709F04CC086
:104A20001A2F0B2F35DB0130B9F41A2F0B2F4EDB69
:104A3000F801EA53F64F00810A1900831A2F0B2F51
:104A400045DBF801EA53F64F00810E94390E01E080
:104A50000093CA0C0C94212E023011F00C94212EDC
:104A60001A2F0B2F33DBF801EA53F64F0081118127
:104A70000F7F13702A2D30E00217130710F40C94E7
:104A8000212E8A2D90E01A2F0B2F20DBF801EA53FC
:104A9000F64F00811181081B190B008311831A2F17
:104AA0000B2F63DBBB2319F40A2F0E94243801E08B
:104AB0000093CA0C0C94212E9DDA903360F09B3742
:104AC00050F4092F0E94810D98A721E08E01085D06
:104AD0001F4F86D905C020E08E01085D1F4F80D989
:104AE00000E00883AE01485D5F4F9E012C593F4FA7
:104AF0008E010E94441D902F992311F40C94212EB5
:104B000023E935E08E010E94221D002351F001E0CF
:104B100000935209A0E0BA2F1A2F0B2F3DDA0C9404
:104B2000212E2FE835E08E010E94221D002351F036
:104B300000E000935209A0E0BA2F1A2F0B2F2CDAB5
:104B40000C94212E2BE336E08E010E94221D0023BF
:104B500041F04BDCA0E0BA2F1A2F0B2F1DDA0C947A
:104B6000212E27E336E08E010E94221D002339F416
:104B700027ED35E08E010E94221D002391F0E3EF26
:104B8000F5E11491EAEEF5E104910E946A2E0E948B
:104B9000D60E2BDCA0E0BA2F1A2F0B2FFDD90C94C8
:104BA000212E22E336E08E010E94221D0023B1F067
:104BB000933021F002E0CCD90C94212EFE01FF9617
:104BC00005A116A127A130A5B02FFE01FF9601A5D2
:104BD00012A523A534A5A02F0C94212E2DE236E09A
:104BE0008E010E94221D002339F42BE236E08E0153
:104BF0000E94221D002341F1E8ECFCE0208131817C
:104C00002F3700E03007E8F4E8ECFCE00081118188
:104C10000F5F1F4F00831183F4DA002341F0E5DBBF
:104C2000A0E0BA2F1A2F0B2FB7D90C94212EE8EC45
:104C3000FCE00081118101501040008311830C942D
:104C4000212E01E085D9FDC724E236E08E010E94C5
:104C5000221D002339F422E236E08E010E94221D3B
:104C6000002321F1E8ECFCE000811181012BD9F057
:104C7000E8ECFCE0008111810150104000831183B9
:104C8000C0DA002339F0B1DBA0E0BA2F1A2F0B2FC6
:104C900083D9D7C7E8ECFCE0008111810F5F1F4F7B
:104CA00000831183CEC701E053D9CBC72DE136E095
:104CB0008E010E94221D002339F42BE136E08E0183
:104CC0000E94221D002399F1923019F002E040D990
:104CD000B8C7FE01FF9605A116A127A130A500388F
:104CE00040E0140740E0240740E03407E8F4E8EC33
:104CF000FCE080819181FE01FF9605A116A127A10C
:104D000030A5E8ECFCE0008311837BDA002339F066
:104D10006CDBA0E0BA2F1A2F0B2F3ED992C7E8EC1C
:104D2000FCE0808391838DC701E012D98AC726E118
:104D300036E08E010E94221D0023D1F1923019F03D
:104D400002E006D97EC7FE01FF9605A116A127A1A4
:104D500030A5003840E0140740E0240740E0340765
:104D600020F5E8ECFCE080819181FE01FF9605A131
:104D700016A127A130A5E8ECFCE00083118341DAFD
:104D8000002371F0E8ECFCE0808391832EDBA0E04F
:104D9000BA2F1A2F0B2F00D901E00093CA0C51C76C
:104DA000E8ECFCE0808391834CC701E0D1D849C78F
:104DB00028E436E08E010E94221D0023E1F00091DC
:104DC000CA0C002389F000E0C3D80E94B20E902FD5
:104DD000993519F0993709F034C704E110E00E94C1
:104DE000580C08E001BD2DC704E110E00E94580CEA
:104DF00008E001BD26C721E136E08E010E94221D98
:104E0000002319F10AE30E94810D20E08E01085D64
:104E10001F4F0E94F01E002361F000E00DAB9E01C9
:104E2000285D3F4F06EC19E00E940A1D01E0009347
:104E3000CA0CE4EFF5E11491EBEEF5E104914AD7E9
:104E400006EC19E00E94A50EFCC62EE036E08E01AD
:104E50000E94221D002309F482C09130A9F580E050
:104E60008F3108F0EEC602E0809F00E0000E02E005
:104E7000101EF001EA53F64F018105FF23C090E0B8
:104E8000FC01E55AF64F00810023E1F021E018E132
:104E9000082F0E949D4A14E2082FF0D622E0829F3C
:104EA00020E0020E22E0121EF001EA53F64F0083CA
:104EB0001183082F0E942438182F00E04FDA182F92
:104EC00000E053D98395CCCF44245524E92FF0E05A
:104ED00031974E165F060CF0B4C6FE01EC59FF4F39
:104EE000042D10E0000F111F000F111FE00FF11F24
:104EF0000081118122813381802F02E0809F00E0B8
:104F0000000E02E0101EF001EA53F64F018105FF8A
:104F100024C0082F10E0F801E55AF64F0081002365
:104F2000E1F021E018E1082F0E949D4A14E2082FC9
:104F3000A5D622E0829F20E0020E22E0121EF001A0
:104F4000EA53F64F00831183082F0E942438182F4C
:104F500000E004DA182F00E008D94394B6CF2AE025
:104F600036E08E010E94221D002309F460C09130BA
:104F700021F580E08F3108F064C690E0FC01E55A2D
:104F8000F64F00810023B9F020E018E1082F0E94BD
:104F90009D4A02E0809F00E0000E02E0101EF0013A
:104FA000EA53F64F018100620183182F00E0D6D941
:104FB000182F00E0DAD88395DDCF44245524E92F5B
:104FC000F0E031974E165F060CF03BC6FE01EC593F
:104FD000FF4F042D10E0000F111F000F111FE00FF5
:104FE000F11F0081118122813381802F082F10E071
:104FF000F801E55AF64F00810023B9F020E018E1EE
:10500000082F0E949D4A02E0809F00E0000E02E00F
:10501000101EF001EA53F64F018100620183182F40
:1050200000E09CD9182F00E0A0D84394C7CF22E01D
:1050300036E08E010E94221D002309F448C0009131
:10504000EE0C1091ED0C011709F0FBC508EC10E017
:105050000E94580C0E94FA1FE3EFF5E11491EAEE6A
:10506000F5E1049137D612E205E60E94784A0E94E3
:10507000390E00E20E94810D13E205E60E94784A93
:105080000E94390E00E20E94810D14E205E60E94A2
:10509000784A0E94390E0CE20E94810D12E206E667
:1050A0000E94784A0E94390E00E20E94810D13E2AC
:1050B00006E60E94784A0E94390E00E20E94810DA5
:1050C00014E206E60E94784A0E94390EB8CF23E81F
:1050D00036E08E010E94221D002339F421E836E0DB
:1050E0008E010E94221D0023C1F0FE01FF9605A142
:1050F00016A127A130A5923021F002E00E94A81F3E
:10510000A0C5083020F004E00E94A81F9AC50093B3
:10511000DA0901E00093CA0C94C52CE736E08E0151
:105120000E94221D002399F1933021F002E00E9499
:10513000A81F87C5FE01FF9605A116A127A130A5CE
:10514000802FFE01FF9601A512A523A534A5902F5F
:10515000983010F4883020F004E00E94A81F71C538
:105160000AE30E94810D082F0E94390E0DE20E9471
:10517000810D0EE30E94810D092F0E94390E182F18
:10518000092F0E94471F01E00093CA0C5AC528E767
:1051900035E08E010E94221D002341F423E735E013
:1051A0008E010E94221D002309F488C0933020F054
:1051B00002E00E94A81F45C5913019F40091DA0958
:1051C00006C0FE01FF9605A116A127A130A5073054
:1051D00020F004E00E94A81F34C5E8ECFCE0208128
:1051E0003181232B41F41091DA09133020F004E0CF
:1051F0000E94A81F26C5923039F417E00E94471F6D
:1052000001E00093CA0C19C09130A1F40091DA09B1
:10521000073080F417E00091DA090E94471FE6EC9E
:10522000F9E004890395048B0E94152001E00093A6
:10523000CA0C03C004E00E94A81FE8ECFCE0008157
:105240001181012B09F0FDC40091DA09013029F028
:105250000091DA09023009F0F4C400E410E020E81B
:1052600030E040EC50E080E01EC062E0869F020E1D
:10527000131EF001EA53F64F2080318062E0869FD2
:10528000000E111EF001EA53F64F60817181261A5B
:10529000370A62E0869F040E151EF001EA53F64FAE
:1052A0002082318283958F3100F30E94FA1F03E040
:1052B0000E94A81F02E00E947A1FC3C425E736E0BF
:1052C0008E010E94221D002339F42BEF35E08E0160
:1052D0000E94221D0023E9F1923029F5FE01FF967C
:1052E00005A116A127A130A5802F873020F004E06A
:1052F0000E94A81FA6C40091DA09801770F4E6EC9A
:10530000F9E004890A95048B0E94152006C0182F25
:105310001395082F0E94471F83958630C0F301E044
:105320000093CA0C8EC4913009F08BC40091DA0945
:10533000013058F0E6ECF9E004890A95048B0E94EC
:10534000152001E00093CA0C7CC404E00E94A81F51
:1053500078C42EE636E08E010E94221D002339F427
:105360002CE636E08E010E94221D002389F1FE0109
:10537000FF9605A116A127A130A5802F923021F01C
:1053800002E00E94A81F5DC4873020F004E00E9464
:10539000A81F57C406E0402E06C0142D1A95042DF0
:1053A0000E94471F4A948415C0F317E0082F0E94FB
:1053B000471F0091DA09801738F4E6ECF9E0048918
:1053C0000395048B0E94152001E00093CA0C39C498
:1053D00025EB35E08E010E94221D002379F09230EA
:1053E00048F0FE01FF9605A116A127A130A50E9455
:1053F000BC3E27C401E00E94BC3E23C42AE435E041
:105400008E010E94221D002341F428E435E08E0124
:105410000E94221D002309F461C0FE01FF9605A130
:1054200016A127A130A5402E923021F002E00E9463
:10543000A81F07C407E0401620F004E00E94A81F40
:1054400000C499E580E01DC0082F10E0F801E55A7E
:10545000F64F00810023A1F0042D10E040E450E05D
:105460000E94EE4A22E0829F000E111E00E4000E10
:1054700000E0101EF001EA53F64F018106FD9EE4A4
:1054800083958F3108F30091DA09401640F0993581
:1054900031F400E00E94A81F0E94B20E902F9935AF
:1054A00019F0993709F0CDC3E8EFF5E11491EFEE6B
:1054B000F5E104910FD4042D0E94390E07E00E94FB
:1054C0007A1F142D07E00E94471F80E08F3108F0FB
:1054D000B8C3082F0E9424388395F8CF27E636E01A
:1054E0008E010E94221D002309F4B0C0E8ECFCE00C
:1054F00040805180913061F4E8ECFCE00081118142
:1055000020E030E0FE01FF9605A316A327A330A7F5
:10551000E5EAFDE020813181273302E0300738F0F1
:1055200023E333E012E20EEF0E94A54A06C02FEFFC
:1055300033E012E20EEF0E94A54A00E010E0E8EC32
:10554000FCE00083118380E00CC022E0829F20E019
:10555000020E22E0121EF001EA53F64F008311837F
:1055600083958F3100F590E0FC01E55AF64F0081FC
:105570000023B1F318E1082F0E94784A013021F48A
:105580001EE1082F7BD303C014E2082F77D300302D
:1055900020E41207D1F60DED1DE00E94EB48082F24
:1055A0000E94390EDDCFE8ECFCE040825182FE0122
:1055B000FF9605A116A127A130A59CD411C000918A
:1055C000EE0C1091ED0C011759F00E94B20E0B3148
:1055D00039F401E00093CB0C05EF1DE00E94EB488D
:1055E0000091CD0C002359F700E115E10E94EB4832
:1055F00004EF11E00E94580C80E00CC022E0829F72
:1056000020E0020E22E0121EF001EA53F64F008362
:10561000118383958F31B0F490E0FC01E55AF64F89
:1056200000810023B1F31EE1082F28D3003020E4CD
:10563000120721F70DED1DE00E94EB48082F0E9494
:10564000390EE7CF07E00E947A1FFBC223E636E05F
:105650008E010E94221D002309F457C0923051F49C
:10566000FE01FF9605A116A127A130A5003024E078
:10567000120720F002E00E94A81FE3C21A2F0B2F8E
:105680000E94AE211A2F0B2F0E9448200130E9F40E
:10569000FE01FF9605A116A127A130A5802F1A2F84
:1056A0000B2F0E946620F801EA53F64F80831A2FD1
:1056B0000B2F0E946620F801EA53F64F00810E94EA
:1056C000390E01E00093CA0CBCC2023009F0B9C225
:1056D000FE01FF9605A116A127A130A5C8011A2F2A
:1056E0000B2F0E946620F801EA53F64F80839183C6
:1056F0001A2F0B2F0E94B520BB2319F40A2F0E94EA
:10570000243801E00093CA0C9CC22CE536E08E01DF
:105710000E94221D002341F42AE536E08E010E94FA
:10572000221D002309F443C1BE01605F7F4FEBE2FD
:10573000F8E930E08B0148E150E00E948F4B923055
:1057400071F4FE01FF9605A116A127A130A507302F
:1057500040E0140740E0240740E0340720F002E076
:105760000E94A81F6EC201E00093CA0CFE01FF96C2
:1057700005A116A127A130A5102F07E00E94471F01
:1057800040E452EE60E070E080E03AC002E0809FCA
:105790008001212F220F220B322F040F151F261FED
:1057A000371F0F5F1F4F2F4F3F4FF801322F3BBF67
:1057B000069000E00BBF302C222402E0809F800185
:1057C000212F220F220B322F040F151F261F371FE8
:1057D000F801322F3BBF0690202D00E00BBF30E0D8
:1057E000220D331D2F7F3370FE01E55CFE4F082F25
:1057F00010E0000F111FE00FF11F2083318383950C
:105800008F3120F2FE01FF9605A116A127A130A538
:1058100040E450E00E94EE4A005C1F4F80E026C04A
:1058200022E0829F000E111E21E0020E20E0121ED7
:10583000F001EA53F64F508140E022E0829F000ED3
:10584000111EF001EA53F64F208130E0240F351F7E
:105850002F7F3370FE01E350FF4F482F50E0440F7D
:10586000551FE40FF51F2083318383958F31C0F2DC
:1058700080E068C0FE01E55CFE4F082F10E0000FDD
:10588000111FE00FF11F208131812F7F33708E01B6
:1058900003501F4FFE01709690E0E80FF91F408102
:1058A00050E0440F551F040F151FE02FF12F00810A
:1058B00011810F7F1370201B310B8E01055C1E4F71
:1058C000FE01709690E0E80FF91F408150E0440F10
:1058D000551F040F151FE02FF12F008111810F7F3D
:1058E0001370020F131F22E0829F20E0020E22E0BD
:1058F000121EF001EA53F64F008311838E0103500C
:105900001F4FFE01709690E0E80FF91F208130E0F4
:10591000220F331F020F131FE02FF12F008111817F
:1059200000701C7F22E0829F20E0020E22E0121E07
:10593000F001EA53F64F20813181202B312B208357
:10594000318383958F3138F590E0FC01E55AF64FAD
:1059500000810023B1F3FE01709690E0E80FF91F7B
:1059600000810F3F09F086CFFE01E350FF4F082F63
:1059700010E0000F111FE00FF11F0081118122E0E4
:10598000829F20E0020E22E0121EF001EA53F64F41
:1059900000831183D6CF07E00E947A1F80E08F3109
:1059A00008F04FC1082F0E9424388395F8CF26E5D0
:1059B00036E08E010E94221D0023C1F000E00E940B
:1059C000A81F0E94B20E093519F0093709F039C134
:1059D0000E9470210E94F521A0E0BA2F1A2F0B2FF0
:1059E0000E94CC1F01E00093CA0C2BC121E536E0D8
:1059F0008E010E94221D002341F42DE436E08E0129
:105A00000E94221D002309F418C110E088242FEF02
:105A10003FE0A9010E94D04A22EF3FE0A9010E9485
:105A2000DC4A01E12FEF3FE0A9010E94DC4A80E05F
:105A300090E006C0FC01EA53F64F0081100F01967A
:105A4000803002E09007B0F30091E509011B0A9550
:105A50000093E5090EE20E94810D80E090E00BC00A
:105A6000FC01EA53F64F00819C012050384FA901F8
:105A70000E94DC4A0196803002E0900788F3009192
:105A8000040C20E03AE0A9010E94DC4A0091050CD8
:105A900021E03AE0A9010E94DC4A80E090E001C0E8
:105AA0000196803002E0900770F49C012050384F3E
:105AB000A9010E94D04AFC01EA53F64F1081011758
:105AC00079F388248394E8ECFCE00081118125EFD0
:105AD0003FE0A9010E94DC4A882009F075C025EF4B
:105AE0003FE0A9010E94D04AE8ECFCE0208131812E
:105AF000021709F069C00AEA24EF3FE0A9010E94F9
:105B0000DC4A08E001BD04EF11E00E94580C25EFCB
:105B10003FE0A9010E94D04A10E0E8ECFCE00083DD
:105B20001183E8ECFCE0008111810F7F107000838D
:105B3000118388240FEF24EF3FE0A9010E94DC4A83
:105B4000E8ECFCE00081118120E030E040E052E030
:105B500060E070E00E942F4B2801390100E0400E08
:105B600000EE501E00E0601E00E0701E80E090E03D
:105B700001C00196803002E09007C0F49C012050E3
:105B8000384FA9010E94D04A602F8C0120E030E0FC
:105B9000040D151D261D371DF801322F3BBF069041
:105BA00000E00BBF601529F302E0802E20E03AE010
:105BB000A9010E94D04A0093040C21E03AE0A90117
:105BC0000E94D04A0093050C8820F9F40E9401211C
:105BD0000091DB09002361F0E8ECFCE00081118119
:105BE0002091DB0930E020503F4FA9010E94DC4AA0
:105BF00000E115E10E94EB480E94F521A0E0BA2FD8
:105C00001A2F0B2F0E94CC1F09C005ED1DE00E942A
:105C1000EB4800E3800E082D0E94810D00E0009308
:105C2000CA0C22EF3FE0A9010E94D04A2FEF3FE0CB
:105C3000A9010E94DC4AAD9804C008EE1DE00E9454
:105C4000EB480091DA09091599F00091DA09013F52
:105C500020F000E00093DA0907C00091DA0908306B
:105C600018F007E00093DA090E9415209090DA09F5
:105C70001A2F0B2F0E94AE210C9497239A938A938C
:105C8000802F082F0E94874A0F3F2FEF120719F429
:105C900000E012E01CC0E8ECFCE020813181232B05
:105CA00051F090E0880F991FFC01EA57F64F2081D0
:105CB0003181021B130B212F27FF03C000E010E0EE
:105CC00006C0003024E0120710F00FEF13E08991B6
:105CD000999108959A938A93902F812F02E00E94C0
:105CE000810D0BE10E94810D0BE50E94810D8A3030
:105CF00038F0082F4AE00E94E04A005D0E94810DC2
:105D0000082F4AE00E94E04A042F005D0E94810DA6
:105D10000BE30E94810D9A3038F0092F4AE00E946F
:105D2000E04A005D0E94810D092F4AE00E94E04A8E
:105D3000042F005D0E94810D06E60E94810D89916D
:105D4000999108959A938A93FA93EA933A922A92B0
:105D50001A920A927A936A935A934A933A932A939D
:105D60001A930A938FB79BB700E00BBF789400910A
:105D7000CD0C002349F00091CC0C002321F004E26B
:105D80000E94810D01C0D2D0EFEDFCE000811181B5
:105D90000F5F1F4F008311830091EC0D102F13959F
:105DA0001093EC0D0F70002309F06EC0E1EEFCE0E3
:105DB00000811181012B41F0E1EEFCE000811181B5
:105DC00001501040008311830091DE0C002349F044
:105DD000EEEDFCE000810A95008308E015B3102782
:105DE00015BBAA9AA99A24B135B10091AD0D10E066
:105DF00003701070000F111FF801EB55F24F208354
:105E00003183EDEAFDE0008103950083037007B95B
:105E10000091ED0D102F13951093ED0D07700023D9
:105E200099F5ECE9FDE00081039500830E9418419B
:105E3000879B2AC0969B28C00091D80C002321F58F
:105E400000919A000F7700939A00959A96980FE127
:105E500013E001501040E9F700C0000000919B00E2
:105E6000102F17FF0AC000919C00053531F404E1A2
:105E700010E00E94580C08E001BD969A9598009198
:105E80009A00006800939A00EEEAFDE0008107FFA7
:105E90000CC00091EC0D002311F4A89815C00091DE
:105EA000EC0D083089F4A89A0FC00091EC0D109108
:105EB000AE0D1023112341F40091AE0D002321F00B
:105EC00001E015B3102715BB00E00093000D9BBF48
:105ED0008FBF0991199129913991499159916991EE
:105EE00079910990199029903990E991F9918991C6
:105EF000999118959A938A93C80120E030E010E2B6
:105F00000EEF0E94A54AEAEDFCE080839183ECED60
:105F1000FCE08083918301E00093D90C0093CD0CC9
:105F200000E00093CB0C8991999108950E94A04BB9
:105F300024970091D90C002309F44DC000E0009390
:105F40002F1000E010E0E5E2F0E100831183E3E2CE
:105F5000F0E100831183E7E2F0E10083118300E0C8
:105F60000093960C03E000932D10CC2431C002E086
:105F7000C09E800100501E4FF801EA53F64F208169
:105F800031810C2D10E0000F111FF801E650F14F88
:105F90002083318300E010E02C2D30E0220F331FEE
:105FA000F901E054F04F008311832C2D30E0220FD3
:105FB000331FF901EE50F24F008311832C2D30E096
:105FC000220F331FF901E258F04F00831183C3946D
:105FD0000FE1C01660F2E3E2F0E100811181E5E239
:105FE000F0E1208131810217130708F064C2E3E277
:105FF000F0E1008111810F5F1F4F00831183009139
:106000002D10033009F457C280E00CE190E0FC0150
:10601000E857F84F0083839504E090E0FC01E857CF
:10602000F84F00838395CC246EC002E0C09E00E050
:10603000000E02E0101EF001EA53F64F208131817C
:10604000203004E0300768F00FEF13E022E0C29E3A
:1060500020E0020E22E0121EF001EA53F64F008308
:10606000118390E0FC01E857F84FC082839501E06E
:1060700010E02C2D30E0205E3F4FF901E957F34F3F
:10608000408142954F700E94FE4A90E0FC01E85723
:10609000F84F0083839501E010E02C2D30E0205E66
:1060A0003F4FF901E957F34F40814F700E94FE4A7C
:1060B00090E0FC01E857F84F0083839502E0C09E12
:1060C00000E0000E02E0101EF001EA53F64F0081DE
:1060D000118190E0FC01E857F84F0083839502E0BE
:1060E000C09E00E0000E02E0101EF001EA53F64FE1
:1060F00000811181012F10E090E0FC01E857F84F7A
:1061000000838395C3940FE1C01608F0C8C1DD2455
:10611000F601E55AF64F00810023A1F300912D10FE
:10612000002309F092C00C2D10E0000F111FF801A0
:10613000E45CF04F008111812C2D30E0220F331FE1
:10614000F901E258F04F20813181021B130B212FFE
:10615000220F220B322FE3E2F0E14081518160E017
:1061600070E00E942F4BE5E2F0E14081518160E058
:1061700070E00E94794B2C2D30E0220F331FF90183
:10618000E258F04F40815181400F511F2C2D30E0DB
:10619000220F331FF901E054F04F408351832C2D1F
:1061A00030E0220F331FF901E258F04F2081318196
:1061B00015950795020F131F212F220F220B322F47
:1061C000E3E2F0E14081518160E070E00E942F4BFA
:1061D00040E950E060E070E00E942F4B4FE050E05B
:1061E00060E070E00E94794B012F122F232F330FB4
:1061F000330B2595179507952C2D30E0220F331F73
:10620000F901EA58F14F008311830C2D10E0000FC3
:10621000111FF801E854F14F208131810C2D10E05D
:10622000000F111FF801EA58F14F00811181020F90
:10623000131F22E0C29E20E0020E22E0121EF00197
:10624000EA53F64F0083118310C100912D100130E5
:1062500009F046C00C2D10E0000F111FF801E854A2
:10626000F14FA081B1810C2D10E0000F111FF8013A
:10627000EC5CF14F00811181212F220F220B322F74
:10628000E3E2F0E14081518160E070E00E942F4B39
:10629000E5E2F0E14081518160E070E00E94794BDD
:1062A0000A0F1B1F22E0C29E20E0020E22E0121EF7
:1062B000F001EA53F64F008311830C2D10E0000F1C
:1062C000111FF801E45CF04F208131810C2D10E0AA
:1062D000000F111FF801E054F04F20833183C5C037
:1062E000DD24F601EE5FFF4E0081002309F078C047
:1062F0000C2D10E0000F111FF801E258F04F008143
:106300001181119501951040212F220F220B322F60
:10631000E3E2F0E14081518160E070E00E942F4BA8
:10632000E5E2F0E14081518160E070E00E94794B4C
:106330002C2D30E0220F331FF901E258F04F40813D
:106340005181400F511F2C2D30E0220F331FF901D6
:10635000E054F04F408351832C2D30E0220F331F47
:10636000F901E854F14FA081B1812C2D30E0220FCA
:10637000331FF901E258F04F2081318115950795BF
:10638000020F131F212F220F220B322FE3E2F0E125
:106390004081518160E070E00E942F4B40E950E065
:1063A00060E070E00E942F4B4FE050E060E070E052
:1063B0000E94794B012F122F232F330F330B25957A
:1063C000179507950A0F1B1F22E0C29E20E0020EC0
:1063D00022E0121EF001EA53F64F0083118345C0FC
:1063E0000C2D10E0000F111FF801E854F14FA081AF
:1063F000B1810C2D10E0000F111FF801EC5CF14F82
:1064000000811181212F220F220B322FE3E2F0E1D4
:106410004081518160E070E00E942F4BE5E2F0E1A5
:106420004081518160E070E00E94794B0A0F1B1F90
:1064300022E0C29E20E0020E22E0121EF001EA538A
:10644000F64F008311830C2D10E0000F111FF8018F
:10645000E45CF04F208131810C2D10E0000F111F02
:10646000F801E054F04F2083318302E0C09E00E049
:10647000000E02E0101EF001EA53F64F018107FF03
:10648000D4CD00E010E022E0C29E20E0020E22E027
:10649000121EF001EA53F64F00831183E2CD282F3C
:1064A00013E80EEF0E94534700912F10002319F0BC
:1064B00000E00093CD0CE3E2F0E100811181E5E220
:1064C000F0E1208131810217130708F4B9C500E01B
:1064D00010E0E3E2F0E100831183CC2427C002E066
:1064E000C09E00E0000E02E0101EF001EA53F64FDD
:1064F000208131810C2D10E0000F111FF801E854AC
:10650000F14F208331830C2D10E0000F111FF80193
:10651000E054F04F208131810C2D10E0000F111F4D
:10652000F801E258F04F20833183C3940FE1C01685
:10653000B0F200912D10002309F09FC001E00093FC
:106540002D10E9E2F0E100811181EBE2F0E1208120
:106550003181220F331F021B130BE5E2F0E10083B0
:106560001183CC2446C00C2D10E0000F111FF80140
:10657000EE50F24F808191810C2D10E0000F111F21
:10658000F801EA58F14F00811181801B910B0C2D0D
:1065900010E0000F111FF801E45CF04F0081118141
:1065A000212F220F220B322FEBE2F0E140815181AB
:1065B00060E070E00E942F4B4CE050E060E070E043
:1065C0000E942F4B45E050E060E070E00E94794B64
:1065D000012F122F232F330F330B801B910B0C2D08
:1065E00010E0000F111FF801EC5CF14F80839183E4
:1065F000C3940FE1C01608F0D6C0DD24F601EE5FAB
:10660000FF4E0081013009F0AECF0C2D10E0000FDD
:10661000111FF801EE50F24F008111812C2D30E056
:10662000220F331FF901EA58F14F20813181021BFB
:10663000130B212F220F220B322FE5E2F0E14081D4
:10664000518160E070E00E942F4BE9E2F0E140816F
:106650005181EBE2F0E160817181461B570B60E0F4
:1066600070E00E94794B2C2D30E0220F331FF9018E
:10667000EC5CF14F00831183BBCF00912D100130F2
:10668000D1F502E000932D10EBE2F0E100811181E1
:10669000E5E2F0E100831183CC240FE1C01608F09D
:1066A00082C00C2D10E0000F111FF801EE50F24FC8
:1066B000208131810C2D10E0000F111FF801EC5CDE
:1066C000F14F00811181201B310B0C2D10E0000FC8
:1066D000111FF801EA58F14F00811181201B310B85
:1066E0000C2D10E0000F111FF801EC5CF14F20831E
:1066F0003183C394D2CF00912D100230B1F4E7E280
:10670000F0E100811181012B61F003E000932D1075
:10671000E7E2F0E100811181E5E2F0E1008311831D
:1067200042C000E000932D103EC000912D100330B8
:10673000D1F5CC2432C002E0C09E00E0000E02E0A1
:10674000101EF001EA53F64F208131810C2D10E02C
:10675000000F111FF801E650F14F2083318300E054
:1067600010E02C2D30E0220F331FF901E054F04FE0
:10677000008311832C2D30E0220F331FF901EE50DE
:10678000F24F008311832C2D30E0220F331FF901CB
:10679000E258F04F00831183C3940FE1C01658F202
:1067A00000E000932D1000912D10002309F048C443
:1067B000EEE2F0E100810395008300912E1010912C
:1067C0009B0C011728F40091D90C002309F4DEC0BA
:1067D0000091D90C002391F50091960C002329F02B
:1067E000E7E8FCE007850A9507870091960C0023EF
:1067F00029F50091CB0C002339F000E010E0EAED20
:10680000FCE0008311831AC0E0EDFCE000811181FF
:10681000EEECFCE0208131810217130741F000917A
:10682000A10C10E0EAEDFCE00083118307C00091A9
:10683000A00C10E0EAEDFCE000831183EAEDFCE03F
:1068400000811181012B21F401E000932F109EC0E3
:1068500000E00093D90CE8ECFCE000811181EAED46
:10686000FCE0208131810217130741F500E010E0C0
:1068700020E030E0EEEEFDE00083118322833383DD
:106880000091960C002309F053C0ADE0B0E0A034B5
:1068900000E0B00708F04CC0EEEEFDE00081118191
:1068A000228133810A0F1B1FF801EA53F64F008142
:1068B000FD01E957F34F00831196E9CFEAEDFCE0C3
:1068C0000081118120E030E0322F212F102F00E0D5
:1068D000110F221F331F005010422F4F3F4FEEEE7B
:1068E000FDE000831183228333830091960C002303
:1068F000F9F4ADE0B0E018C0EEEEFDE0408151816A
:10690000628173818D0120E030E0040F151F261F86
:10691000371FF801322F3BBF069000E00BBFFD018F
:10692000E957F34F00821196A03400E0B00720F33E
:10693000EEEEFDE00081118122813381005C1F4F6A
:106940002F4F3F4F008311832283338300919B0C91
:10695000083020F400919B0C002381F40BE01DE033
:106960000E94EB48EAEDFCE0008111810E94880E54
:106970000DE50E94810D01E000932F100091960C0F
:10698000002309F429CF00E000932E10A0E0B0E02E
:1069900020C0EEEEFDE00081118122813381A8014B
:1069A000B9014F5F5F4F6F4F7F4FEEEEFDE04083C9
:1069B000518362837383F801322F3BBF069000E05E
:1069C0000BBF8D01005C1D4FF801EA53F64F0082AA
:1069D0001196A03400E0B00758F5E8ECFCE0008127
:1069E0001181EAEDFCE0208131810217130789F65D
:1069F000EEEEFDE00081118122813381F801EA533E
:106A0000F64F20818D01005C1D4FF801EA53F64FCF
:106A10002083EEEEFDE000811181228133810F5F42
:106A20001F4F2F4F3F4F0083118322833383D0CFDB
:106A300000912E100395EAEDFCE080819181109188
:106A40009B0C011708F45DC00091CB0C002339F0BA
:106A500000E010E0EAEDFCE00083118319C0009132
:106A6000960C023028F0EAEDFCE08081918110C0A4
:106A7000E0EDFCE000811181EEECFCE02081318151
:106A80000217130719F08091A10C02C08091A00C8D
:106A900090E0E8ECFCE0008111818017910759F447
:106AA00000E410E020E030E0EEEEFDE00083118332
:106AB0002283338326C0882379F4EEEEFDE0008143
:106AC00011812281338100541040204030400083E6
:106AD00011832283338315C0082F10E020E030E0BB
:106AE000322F212F102F00E0110F221F331F005CC7
:106AF0001F412F4F3F4FEEEEFDE0008311832283B5
:106B00003383A0E0B0E01BC0EEEEFDE04081518198
:106B1000628173818D0120E030E0040F151F261F74
:106B2000371FF801322F3BBF069000E00BBF8D01ED
:106B300000581D4FF801EA53F64F00821196A03419
:106B400000E0B007D0F4E8ECFCE000811181801790
:106B5000D9F6EEEEFDE000811181228133810A0F2A
:106B60001B1FF801EA53F64F20818D0100581D4F7D
:106B7000F801EA53F64F2083E1CF00912F10002354
:106B800009F05EC20091440C10E045E00E94FE4A0C
:106B900040919D0C50E00E940A4BE7E2F0E1008337
:106BA00011830091450C10919D0C019F800145E0DF
:106BB0000E94044BD8010A2F0B2B11F4A1E0B0E086
:106BC00000E010E0CC240EC02C2D30E0220F331F4B
:106BD000F901EE50F24F208131810217130708F4BA
:106BE0008901C3942FE1C21608F0E3C0DD24F60149
:106BF000E55AF64F20812223A1F32C2D30E0220FFD
:106C0000331FF901E650F14F4081518122E0C29ECD
:106C100020E0020E22E0121EF001EA53F64F4083FC
:106C200051832C2D30E0220F331FF901E854F14F2E
:106C30004083518320E030E04C2D50E0440F551F3D
:106C4000FA01EA58F14F2083318322E0C29E20E40A
:106C5000020E22E0121EF001EA53F64F208131812C
:106C60004C2D50E0440F551FFA01EA57F64F408172
:106C70005181240F351F432F47FF03C020E030E030
:106C800006C0203044E0340710F02FEF33E04C2DE5
:106C900050E0440F551FFA01E650F14F40815181F9
:106CA000B901641B750B4C2D50E0440F551FFA01C0
:106CB000EE50F24F608371834C2D50E0440F551F0E
:106CC000FA01E650F14F608171814C2D50E0440F84
:106CD000551FFA01E650F14F2083318342E0C49EF4
:106CE00040E8040E42E0141EF001EA53F64F008023
:106CF00011804C2D50E0440F551FFA01EA57F64F12
:106D000040815181400D511D052E07FE03C040E01A
:106D100050E006C04030E4E05E0710F04FEF53E073
:106D20006217730718F42417350730F02617370752
:106D300028F44217530710F420E001C021E0222379
:106D400091F4E7E2F0E120813181232B61F420917D
:106D50002E1030E0E0919B0CF0E031972E173F07AA
:106D60004CF0882339F420E0DD24F601EE5FFF4E7D
:106D7000208306C021E0DD24F601EE5FFF4E208374
:106D80002C2D30E0220F331FF901EE50F24F4081DD
:106D9000518155230AF018CF2C2D30E0220F331FDC
:106DA000F901EE50F24F208131813195219530402B
:106DB00014CF48E250E00E94EE4AC8018D0143E042
:106DC00050E00E94EE4AA8018C010E940A4BE9E2C1
:106DD000F0E10083118300919F0C10E0EBE2F0E101
:106DE00000831183EBE2F0E100811181000F111F9C
:106DF000E9E2F0E12081318102171307E8F1E8E5CB
:106E0000F9E0008102FF13C00BE50E94810D0091A3
:106E10002E100E946A0D0CE20E94810DE9E2F0E161
:106E2000008111810E94880E0DE50E94810DE9E22A
:106E3000F0E100811181012B39F400E010E0EBE278
:106E4000F0E10083118318C0E9E2F0E100811181D3
:106E50000150104016950795EBE2F0E10083118395
:106E6000EBE2F0E100811181012B31F400E010E050
:106E7000E9E2F0E100831183E9E2F0E100811181B0
:106E800020E030E0000F111F221F331FEBE2F0E182
:106E900080819181A0E0B0E0880F991FAA1FBB1FDD
:106EA000081B190B2A0B3B0B48015901880C991C34
:106EB000AA1CBB1C880E991EAA1EBB1E000F111F08
:106EC000221F331F088319832A833B83082D092936
:106ED0000A290B2929F49924AA24BB248824839401
:106EE000088119812A813B81012B022B032B41F45C
:106EF00001E010E020E030E0088319832A833B831F
:106F0000CC2442C00419150926093709A401B5018A
:106F10000E94794B2C2D30E0220F331FF901E45CE5
:106F2000F04F008311830C2D10E0000F111FF801AA
:106F3000E45CF04F20813181203004E030075CF0C8
:106F40000FEF13E02C2D30E0220F331FF901E45C2A
:106F5000F04F008311830C2D10E0000F111FF8017A
:106F6000E45CF04F2081318121300CEF30075CF47C
:106F700001E01CEF2C2D30E0220F331FF901E45CFF
:106F8000F04F00831183C3940FE1C01608F050C086
:106F90000C2D10E0000F111FF801E258F04F008196
:106FA0001181212F220F220B322FAC01BD010E9433
:106FB0002F4B280139010C2D10E0000F111FF80193
:106FC000EE50F24F00811181212F220F220B322F20
:106FD0000801190140E05AE060E070E08001910191
:106FE0000E942F4B080119014CE050E060E070E076
:106FF000800191010E94794BDD24F601EE5FFF4E86
:107000004081442309F07ECF041915092609370968
:10701000488159816A817B810E94794B2C2D30E017
:10702000220F331FF901E45CF04F008311837BCF03
:10703000EBE2F0E100811181E5E2F0E100831183F0
:107040002496EEE00C94AF4B0E94A84B402E5524A2
:10705000F201E55AF64F0081002309F47EC002E0F8
:10706000409E800100501E4FF801EA53F64F018107
:1070700005FF06C020E018E1042D0E949D4A6DC066
:10708000E8ECFCE000811181012BC9F002E0409E98
:1070900000E0000E02E0101EF001EA53F64F0081FE
:1070A00011810F7F1370242D30E0220F331FF9015F
:1070B000EA57F64FA081B181A00FB11F0DC002E0C9
:1070C000409E00E0000E02E0101EF001EA53F64F71
:1070D000A081B181AF7FB3700B2F07FF03C0A0E089
:1070E000B0E006C0A03004E0B00710F0AFEFB3E0AE
:1070F00014E2042D0E94874A0F3F23E0120758F440
:10710000A017B10720F40A1B1B0BC80106C0CD0154
:10711000801B910B02C008E010E09695879596952C
:107120008795883000E0900710F488E090E00EE149
:10713000009388070A2F00938907AB2FB0E0A09334
:107140008A07082F00938B07892F90E080938C0784
:1071500025E013E0042D0E94CE47E6E00C94B74BE7
:107160000E94AA4BD8010091CD0C002309F041C028
:107170000A2F0B2BF1F1A03800E0B007D0F500E0AA
:1071800010E0E8ECFCE00083118380E00BC022E01B
:10719000829F900120503E4FF901EA53F64F008341
:1071A000118383958F3110F590E0FC01E55AF64F7D
:1071B00000810023B1F318E1082F0E94784A0130C2
:1071C00029F41EE1082F0E943E2E04C014E2082F6D
:1071D0000E943E2E003020E41207C9F60DED1DE09E
:1071E0000E94EB48082F0E946A0DDBCF8D010E94A0
:1071F0007A2FE4E00C94B94B6AC00E94B20E109151
:10720000E40C163018F010E01093E40C2091E40C1C
:1072100030E0F901EB51F34F0083E4EEFCE0108124
:1072200013951083053551F50091E40C0250073099
:1072300008F00A5F10E0F801EB51F34F00810F3FB7
:10724000E9F400E00093E40C0FEF2091E40C30E04F
:10725000F901EB51F34F0083E4EEFCE0008103956C
:10726000008305E52091E40C30E0F901EB51F34F88
:107270000083E4EEFCE00081039500830091E40CC0
:10728000063029F50091E50C0F3F09F50091E60C59
:107290000535E9F40091E70C1091E80C1095011701
:1072A000B1F40091E90C1091EA0C1095011779F4F2
:1072B00001E00093E30C3091E90C20E00091E70C31
:1072C00010E0020F131FE0EDFCE00083118300913A
:1072D000EE0C1091ED0C011709F08FCF08959A93E1
:1072E0008A93C901083C09F08EC0183119F48C0149
:1072F00037DFC4C01A3111F01B3149F5E2EDFCE073
:10730000808391830FEF0E94810D05E50E94810D1E
:10731000E2EDFCE0008111810E94810DE2EDFCE0D4
:107320000081118100950E94810DE2EDFCE0008159
:107330001181012F10E00E94810DE2EDFCE000813F
:107340001181012F10E000950E94810D97C01F311F
:1073500059F4882311F401E001C000E0102F10FD62
:10736000AB9A10FFAB988AC0123281F510E020E092
:1073700030E000E00E94AD0C002309F47FC0E6ED90
:10738000FCE0008111810817190729F010E09C0129
:1073900001E00E94AD0CEAE4F9E0038114810817D2
:1073A000190709F46BC0EAE4F9E083839483082F9A
:1073B00023E030E0A9010E94DC4A892F90E0082FE9
:1073C00024E030E0A9010E94DC4A58C0113229F4BF
:1073D000E1EEFCE08083918351C0153221F48C01F1
:1073E0000E94020E4BC0163251F48C010E94020E14
:1073F0000DE00E94810D0AE00E94810D3FC002E075
:1074000010E895D43BC00436F0F00D36E0F420913E
:10741000CD0C222339F021E02093000D2091000DA6
:107420002223E1F7E4E3F7E1212F30E0E20FF31F3D
:107430002491223021F49C010E94A54A1FC0282FCC
:107440000E949D4A1BC02091CD0C222339F021E0DF
:107450002093000D2091000D2223E1F7ECEFF6E1DF
:10746000212F30E0E20FF31F2491223021F49C0100
:107470000E94A54A03C0282F0E949D4A8991999194
:107480000895083C09F0A4C0183129F4ECEDFCE0A3
:10749000008111810895173229F4EAEDFCE00081A2
:1074A00011810895193121F40091CD0C10E0089557
:1074B0001A3111F01B3129F4E2EDFCE00081118159
:1074C00008951C3111F01D3149F496DE00E000935F
:1074D000E30CE0EDFCE00081118108951E3129F4F8
:1074E0008BDE0091E30C10E008951F3141F405B3E9
:1074F0000695069506950095017010E008951232E4
:10750000A1F510E020E030E000E00E94AD0C002387
:1075100039F1EAE4F9E003811481E6EDFCE0208131
:10752000318102171307E1F0E6EDFCE000811181E3
:10753000EAE4F9E003831483E6EDFCE000811181C5
:1075400023E030E0A9010E94DC4AE6EDFCE0008186
:107550001181012F10E024E030E0A9010E94DC4AF3
:10756000EAE4F9E0038114810895143259F410E03B
:1075700020E030E000E00E94AD0CE4EDFCE0008192
:10758000118108951032B9F400E0809902C00061C1
:1075900011E00C9902C0086011E00D9902C004606E
:1075A00011E00E9902C0026011E00F9902C0016063
:1075B00011E010E00895113229F4E1EEFCE00081C1
:1075C0001181089501E010E8B2D30FEF1FEF089585
:1075D0000436E8F00E36D8F42091CD0C222339F091
:1075E00021E02093000D2091000D2223E1F7E4E338
:1075F000F7E1212F30E0E20FF31F2491223019F43C
:107600000E94874A08950E94784A10E008950F3139
:10761000D8F42091CD0C222339F021E02093000DE5
:107620002091000D2223E1F7ECEFF6E1212F30E06D
:10763000E20FF31F2491223019F40E94874A089523
:107640000E94784A10E0089500E010E008959A93AF
:107650008A93E1E0FDE00081118198012F5F3F4FA7
:10766000E1E0FDE02083318320E030E0005010466F
:107670002F4F3F4FF801322F3BBF0690002D10E0F7
:107680001BBFE1E0FDE0408151819A012F5F3F4F38
:10769000E1E0FDE02083318360E070E0405050463F
:1076A0006F4F7F4FFA01362F3BBF0690202D10E021
:1076B0001BBFE1E0FDE040815181CA010196E1E09C
:1076C000FDE08083918360E070E0405050466F4F52
:1076D0007F4FFA01362F3BBF069010E01BBF0023FF
:1076E00021F4102D022FCDDE4EC0023061F4102D9A
:1076F00030E0220F331FF901E35FF24F2081318127
:10770000022FBFDE40C0013069F4002D10E0000FF1
:10771000111FF801E35FF24F00811181102F022F3A
:10772000B0DE31C00330A9F4002D10E0000F111FAE
:10773000F801E35FF24F00811181102F30E0220F3A
:10774000331FF901E35FF24F20813181022F99DE6F
:107750001AC0043039F4502D40E0022F10E0040F1D
:10776000151F11C0053069F4102D00E030E0200F26
:10777000311F220F331FF901E35FF24F00811181A6
:1077800002C000E010E08991999108950E94AA4BEF
:10779000A801E1E0FDE00081118198012F5F3F4FDA
:1077A000E1E0FDE02083318320E030E0005010462E
:1077B0002F4F3F4FF801322F3BBF0690002D10E0B6
:1077C0001BBFE1E0FDE000801180C0010196E1E017
:1077D000FDE080839183C001A0E0B0E0805090463E
:1077E000AF4FBF4FFC013A2F3BBF0690602D10E01A
:1077F0001BBFE1E0FDE000801180C0010196E1E0E7
:10780000FDE080839183C001A0E0B0E0805090460D
:10781000AF4FBF4FFC013A2F3BBF069010E01BBF9C
:10782000002329F49A01102D062F59DD4BC0023098
:1078300069F49A01102D70E0660F771FFB01E35F7A
:10784000F24F40815181042F4ADD3CC0013071F478
:107850009A01002D10E0000F111FF801E35FF24FB5
:1078600000811181102F062F3ADD2CC00330B1F4B6
:107870009A01002D10E0000F111FF801E35FF24F95
:1078800000811181102F70E0660F771FFB01E35F0D
:10789000F24F40815181042F22DD14C0043021F4C5
:1078A00007E010E044D20EC0053061F4102D00E076
:1078B00070E0600F711F660F771FFB01E35FF24FEF
:1078C00040835183E4E00C94B94BC1DEE3E0FDE07A
:1078D00000831183E1E0FDE00081118198012F5FB9
:1078E0003F4FE1E0FDE02083318320E030E00050B5
:1078F00010462F4F3F4FF801322F3BBF069000E05C
:107900000BBF0092090DA3DEE5E0FDE000831183CB
:107910000091090D002379F4E3E0FDE0008111817D
:10792000E5E0FDE0208131810217130711F401E049
:10793000089500E008950091090D013079F4E5E023
:10794000FDE000811181E3E0FDE02081318102173B
:10795000130710F401E0089500E008950091090D67
:10796000023079F4E3E0FDE000811181E5E0FDE023
:10797000208131810217130710F001E0089500E023
:1079800008950091090D033079F4E3E0FDE00081F2
:107990001181E5E0FDE0208131810217130710F429
:1079A00001E0089500E008950091090D043079F494
:1079B000E5E0FDE000811181E3E0FDE0208131811F
:1079C0000217130710F001E0089500E008950091F8
:1079D000090D053079F4E3E0FDE000811181E5E077
:1079E000FDE0208131810217130711F001E00895B5
:1079F00000E0089505E010E09AD100E008950091BC
:107A00000A0D013061F400910C0D002331F000915A
:107A10000B0D002311F001E0089500E0089500919E
:107A20000A0D023061F400910C0D002321F4009145
:107A30000B0D002311F001E0089500E0089506E029
:107A400010E075D100E008959A938A930230C9F04E
:107A5000E1E0FDE0408151819A012F5F3F4FE1E07D
:107A6000FDE02083318360E070E0405050466F4F6E
:107A70007F4FFA01362F3BBF069010E01BBF0092EC
:107A8000080D1091080D1F5F09F440C1125091F0CC
:107A90001A9509F11A9509F44CC01A9509F4F2C027
:107AA0001A9509F4FBC01A9509F407C11A9509F44F
:107AB0001CC137C1002331F0CADDE1E0FDE00083E5
:107AC000118332C1E1E0FDE0008111810D5F1F4FA4
:107AD0000083118329C1002319F1E1E0FDE0008159
:107AE00011810D5F1F4F00831183B1DDE5E0FDE0E3
:107AF00000831183E1E0FDE0008111810650104018
:107B000000831183E5E0FDE0008111813FDEE1E0CB
:107B1000FDE0008111810D5F1F4F0083118304C1BF
:107B2000E1E0FDE0008111810A5F1F4F00831183B6
:107B3000FBC0002309F49DC0E1E0FDE0008111815C
:107B40000D5F1F4F0083118382DDE3E0FDE00083C2
:107B50001183E1E0FDE00081118198012F5F3F4F2B
:107B6000E1E0FDE02083318320E030E0005010466A
:107B70002F4F3F4FF801322F3BBF069000E00BBF65
:107B80000092090D64DDE5E0FDE0008311830091C2
:107B9000090D002359F4E3E0FDE000811181E5E0E7
:107BA000FDE080819181800F911F50C00091090DEF
:107BB000013059F4E3E0FDE080819181E5E0FDE0F2
:107BC00000811181801B910B41C00091090D023091
:107BD00061F4E3E0FDE000811181E5E0FDE040813A
:107BE00051810E94EE4AC80131C00091090D033055
:107BF00061F4E3E0FDE000811181E5E0FDE040811A
:107C000051810E940A4BC80121C00091090D003129
:107C100059F4E3E0FDE000811181E5E0FDE08081C1
:107C200091818023912312C00091090D013159F4F3
:107C3000E3E0FDE000811181E5E0FDE080819181DC
:107C4000802B912B03C004E010E071D0E1E0FDE057
:107C5000008111810A501040008311838C0196DD50
:107C6000E1E0FDE000811181095F1F4F0083118376
:107C70005BC0E1E0FDE000811181065F1F4F0083E2
:107C8000118352C0002309F04FC0E1E0FDE0008104
:107C90001181E1E0FDE00083118346C0002321F063
:107CA0000BE10093070D40C0E1E0FDE00081118190
:107CB000E1E0FDE00083118337C0002369F0E1E0DB
:107CC000FDE0008111810D5F1F4F61D2C0DCE1E05A
:107CD000FDE00083118328C0E1E0FDE00081118117
:107CE0000D5F1F4F008311831FC0002331F079D235
:107CF000E1E0FDE00083118317C0E1E0FDE00081D9
:107D00001181E1E0FDE0008311830EC0002361F4E6
:107D1000E1E0FDE000811181E1E0FDE000831183FD
:107D200003C003E110E003D08991999108959A93DB
:107D30008A93C801E8E5F9E0008101FF1AC003E574
:107D400015E10E94EB488C010E94880E0BE50E9411
:107D5000810DE1E0FDE0008111810E94880E0AE3BF
:107D60000E94810D0091080D0E946A0D0DE50E9490
:107D7000810D8991999108950E94AB4BA02FAA2360
:107D800011F49598969A00E010E0E1E0FDE00083A0
:107D9000118380E090E204E00093080DAA2321F013
:107DA00004E115E10E94EB4800E00093070D05C0D7
:107DB00002E04ADEAA2309F013D10091070D0B312E
:107DC00009F407C1E1E0FDE020813181203000ECC1
:107DD000300708F0FEC00091080D053009F4F9C025
:107DE000E1E0FDE0008111810817190708F0F1C0FA
:107DF000E1E0FDE00081118198012F5F3F4FE1E05C
:107E0000FDE02083318320E030E0005010462F4F0A
:107E10003F4FF801322F3BBF069000E00BBF0092AE
:107E2000080DE8E0FDE0008107FFC2CF0091080DDA
:107E3000005849F00A9509F46FC00A9509F4B0C0DA
:107E40000A95B1F1C2C041DD00930B0D00910B0DFD
:107E500000930C0DE1E0FDE00081118198012F5F9E
:107E60003F4FE1E0FDE02083318320E030E000502F
:107E700010462F4F3F4FF801322F3BBF069000E0D6
:107E80000BBF00920A0DAA2309F0AAD000910A0D97
:107E9000002309F092CF00910C0DD6DDAA2309F43E
:107EA0008CCF00910C0D002309F487CF99D085CF9A
:107EB0000CDD00930B0DA3DD00930C0DE1E0FDE064
:107EC0000081118198012F5F3F4FE1E0FDE02083A9
:107ED000318320E030E0005010462F4F3F4FF80133
:107EE000322F3BBF069000E00BBF00920A0DAA2381
:107EF00009F076D000910A0D002309F05ECF0091C1
:107F00000C0DA2DDAA2309F458CF00910C0D00231B
:107F100009F453CF65D051CF00910C0D002359F0D7
:107F2000E1E0FDE000811181085F1F4F00831183B4
:107F300000E08ADD42CFC9DC00930B0D00910B0DF0
:107F400000930C0DE1E0FDE00081118198012F5FAD
:107F50003F4FE1E0FDE02083318320E030E000503E
:107F600010462F4F3F4FF801322F3BBF069000E0E5
:107F70000BBF00920A0DAA2309F032D000910A0D1E
:107F8000002309F01ACF00910C0D5EDDAA2309F43D
:107F900014CF00910C0D002309F40FCF21D00DCF89
:107FA000AA2309F01DD000910C0D002311F401E06B
:107FB00001C000E049DDAA2309F4FFCE00910C0DB9
:107FC000002309F0FACE0CD0F8CE00E110E0AFDECD
:107FD000F4CE0091CD0C0023E1F7E3E00C94BA4B12
:107FE0000CE810E00E94EB4866D00DE20E94810D83
:107FF0000091080D0E946A0D0AE30E94810D00E2C3
:108000000E94810D00910B0D0E946A0D0DE30E94EC
:10801000810D08E20E94810DE3E0FDE00081118105
:108020000E94880E0CE20E94810D00E20E94810DE8
:108030000091090D0E946A0D0CE20E94810D00E280
:108040000E94810DE5E0FDE0008111810E94880E13
:1080500009E20E94810D00E20E94810D00910A0D4B
:108060000E946A0D0BE70E94810D00910C0D0E9489
:108070006A0D0DE70E94810D0BE50E94810DE1E084
:10808000FDE0008111810E94880E0DE50E94810DA6
:108090000E94B20E0093070D0091070D0B3151F4B1
:1080A00006E415E10E94EB48E1E0FDE0008111816A
:1080B0000E94880E08950091080D003829F40DE5FE
:1080C00015E10E94EB4808950091080D013829F44C
:1080D00005E615E10E94EB4808950091080D02386D
:1080E00029F40DE615E10E94EB4808950091080D72
:1080F000033829F405E715E10E94EB480895009143
:10810000080D013029F40DE715E10E94EB480895B0
:108110000091080D023029F405E815E10E94EB48B2
:1081200008950091080D033029F40DE815E10E942F
:10813000EB4808950091080D043029F405E915E194
:108140000E94EB4808950091080D053029F40DE9CF
:1081500015E10E94EB4808950091080D063029F4BE
:1081600005EA15E10E94EB4808950091080D0730DB
:1081700029F40DEA15E10E94EB4808950091080DDD
:108180000F3F21F405EB15E10E94EB480895209183
:108190009B0D2A3010F520919B0D30E0220F331FEC
:1081A000F901EF58F24F00831183EBE9FDE0008104
:1081B0000395008320910C0D30E000919B0D10E0A1
:1081C000000F111FF801EF58F24F20833183EBE9C4
:1081D000FDE0008103950083089509E010E0A7DD2C
:1081E000089500919B0D0023E9F0EBE9FDE000818B
:1081F0000A95008310E0000F111FF801EF58F24FAD
:108200000081118100930C0DEBE9FDE000810A95DE
:10821000008310E0000F111FF801EF58F24F0081AA
:10822000118108950AE010E082DD0FEF1FEF08953D
:108230000E94AA4B00913010002309F0D3C0009196
:108240005109013009F094C0E5EAFDE00281138193
:10825000012B09F45AC000E000939C0D00E010E0EF
:10826000E1EAFDE00083118300E010E0E1E3F0E1EA
:108270000083118301E000933010E5EAFDE0008106
:10828000118145E050E00E940A4B10E0EDE9FDE06D
:1082900000831183EDE9FDE080819181E5EAFDE055
:1082A0000281138145E050E00E940A4B10E0801BE0
:1082B000910BEFE9FDE080839183EFE9FDE0208100
:1082C0003181243700E0300720F003E00093AE0D49
:1082D0001FC2EFE9FDE020813181223700E0300745
:1082E00020F007E00093AE0D13C2EFE9FDE020811E
:1082F0003181203700E0300720F00FE00093AE0D11
:1083000007C20FE00093AE0D03C200919C0D0370F5
:10831000002309F0FDC1E5EAFDE00081118145E09F
:1083200050E00E940A4B10E0EDE9FDE0008311836C
:10833000EDE9FDE080819181E5EAFDE002811381B4
:1083400045E050E00E940A4B10E0801B910BEFE9E2
:10835000FDE080839183EFE9FDE0208131812935C3
:1083600000E0300708F0D4C10FE70093AE0DD0C194
:10837000E5EAFDE002811381012B09F0C9C10091FA
:108380009C0D0370002309F0C3C1E5EAFDE0008104
:10839000118145E050E00E940A4B10E0EDE9FDE05C
:1083A00000831183EDE9FDE080819181E5EAFDE044
:1083B0000281138145E050E00E940A4B10E0801BCF
:1083C000910BEFE9FDE080839183EFE9FDE02081EF
:1083D0003181293500E0300708F09AC10FE700939A
:1083E000AE0D96C100913010013009F042C1E5EAAE
:1083F000FDE002811381012B61F400E010E01BBD60
:108400000ABD00E00093AE0DA89800E00093301084
:108410007FC100919C0D0F71002329F400E010E052
:108420001BBD0ABD75C100919C0D0F71023009F092
:108430006FC1E5EAFDE00081118145E050E00E9456
:108440000A4B10E0EDE9FDE000831183EDE9FDE06A
:1084500080819181E5EAFDE00281138145E050E0F1
:108460000E940A4B10E0801B910BEFE9FDE0808336
:108470009183E1EAFDE000811181EFE9FDE02081D7
:1084800031810217130740F4EFE9FDE0008111810B
:10849000E1EAFDE000831183ECEFF5E1A9EABDE03C
:1084A0000D911C9111971695079516950795E00F5C
:1084B000F11F049110E0E3EAFDE000831183EFE98E
:1084C000FDE0008111810A5F1F4FEDE9FDE0208191
:1084D00031810217130718F00FEF13E010C00AEFF5
:1084E00017E1EDE9FDE040815181EFE9FDE02081F8
:1084F0003181421B530B465050400E940A4B0030C2
:1085000024E0120710F00FEF13E01BBD0ABDA3EA31
:10851000BDE0ED91FC911197F69720F003E00093F8
:10852000AE0D32C0A3EABDE0ED91FC911197F49736
:1085300020F007E00093AE0D27C0EFE9FDE02081B9
:108540003181243700E0300720F003E00093AE0DC6
:108550001BC0EFE9FDE020813181223700E03007C8
:1085600020F007E00093AE0D0FC0EFE9FDE02081A1
:108570003181203700E0300720F00FE00093AE0D8E
:1085800003C00FE00093AE0DE1E3F0E10081118143
:108590000F5F1F4F00831183E1E3F0E12081318100
:1085A000283601E0300758F000E010E01BBD0ABD9E
:1085B0000FEF0093AE0D02E800933010A9C0EFE971
:1085C000FDE020813181263700E0300758F000E0DF
:1085D00010E01BBD0ABD0FEF0093AE0D01E8009344
:1085E000301096C0E1EAFDE0008111810C5310408B
:1085F000EFE9FDE0208131810217130758F000E018
:1086000010E01BBD0ABD0FEF0093AE0D03E8009311
:1086100030107EC0E3EAFDE0208131812C3300E0A0
:10862000300758F000E010E01BBD0ABD0FEF0093CB
:10863000AE0D04E8009330106BC0A3EABDE0ED91ED
:10864000FC911197F89708F463C0EFE9FDE02081F1
:108650003181203700E0300708F45AC000E010E014
:108660001BBD0ABD0FEF0093AE0D04E80093301060
:108670004FC000915109023041F002E000935109CE
:1086800027E030E0A9010E94DC4AE5EAFDE0028132
:108690001381012BC1F400E010E01BBD0ABD00E016
:1086A0000093AE0DA89800E000933010009151099E
:1086B000002371F100E00093510927E030E0A901A7
:1086C0000E94DC4A25C000919C0D0F71002301F52A
:1086D000E5EAFDE00081118145E050E00E940A4B8F
:1086E00010E0EDE9FDE000831183EDE9FDE080811C
:1086F0009181E5EAFDE00281138145E050E00E94AE
:108700000A4B10E0801B910BEFE9FDE08083918321
:10871000E4E00C94B94B07EE06B900E010E01BBD95
:108720000ABD03EC0FBD02E00EBD03E00093AD0DEA
:10873000EDEAFDE0008103950083037007B901E0D5
:1087400010E00E94580C24B135B10091AD0D10E03D
:1087500003701070000F111FF801EB55F24F2083CA
:108760003183EDEAFDE0008103950083037007B9D2
:1087700001E010E00E94580C24B135B10091AD0D1C
:1087800010E003701070000F111FF801EB55F24F4D
:1087900020833183EDEAFDE00081039500830370BF
:1087A00007B901E010E00E94580C24B135B10091E6
:1087B000AD0D10E003701070000F111FF801EB55A4
:1087C000F24F20833183EDEAFDE0008103950083C1
:1087D000037007B901E010E00E94580C24B135B1D4
:1087E0000091AD0D10E003701070000F111FF80123
:1087F000EB55F24F2083318308950E94AB4B1A98BA
:108800001B9A0E94D40BA89800E00093560900938D
:10881000570900E0009358090093590900E00093BC
:10882000CD0C00E00093DE0C22E030E0A9010E94B4
:10883000D04A0F3FA9F021E030E0A9010E94D04AC0
:108840000F3F71F023EF3FE0A9010E94D04A0330AF
:1088500038F427E030E0A9010E94D04A033048F103
:1088600001E000934B0921E030E0A9010E94DC4ABD
:1088700002E200934A0920E030E0A9010E94DC4AAC
:1088800000E022E030E0A9010E94DC4A80E023EF12
:108890003FE0082FA9010E94DC4A0AE00093DE0CA9
:1088A00000E00093510927E030E0A9010E94DC4A72
:1088B00029C021E030E0A9010E94D04A00934B0971
:1088C00020E030E0A9010E94D04A00934A0923EF3A
:1088D0003FE0A9010E94D04A802F23E030E0A901A7
:1088E0000E94D04A00934D0924E030E0A9010E9483
:1088F000D04A00934E0927E030E0A9010E94D04AF7
:108900000093510900E00093520911E020E830E0A3
:1089100000E00E94B50B21E010914A0900E00E949E
:10892000240C21E012E201E00E94240C00E00093FC
:10893000560900935709EFDE789424EF3FE0A90130
:108940000E94D04A053519F400E060D45EC183303E
:1089500038F080E023EF3FE0082FA9010E94DC4AB5
:1089600094B700E004BF21EF3FE0A9010E94D04A84
:10897000002361F0923051F48395833008F080E059
:1089800023EF3FE0082FA9010E94DC4A9A70992347
:1089900061F400915109002341F000E00093510976
:1089A00027E030E0A9010E94DC4A21EF3FE0A90165
:1089B0000E94D04A013031F001E021EF3FE0A901EF
:1089C0000E94DC4A00915109023009F05DC000E8C4
:1089D000009330100FEF0093AE0D56C090E0809BD7
:1089E00004C002E310E00E94580C0091EE0C1091BC
:1089F000ED0C011769F00E94B20EA02FA53521F4ED
:108A00000091ED0C0093EE0C082F0E94810D01C027
:108A1000A0E0882311F4AC9807C0813011F4AD9820
:108A200003C0823009F4AE98933209F046C0A332F5
:108A300009F043C004E110E00E94580C08E001BDB9
:108A4000809B04C002E310E00E94580C0C991CC0EB
:108A500002E310E00E94580C00915109002371F4C8
:108A6000E5EAFDE002811381012B41F001E0009372
:108A7000510927E030E0A9010E94DC4A0C9BFECF9F
:108A800002E310E00E94580C809B31C0AD9AAC9A72
:108A9000AE9A0091EE0C1091ED0C011709F49ECFE7
:108AA0000E94B20E902F953521F40091ED0C0093A9
:108AB000EE0C082F0E94810D92CF993011F0A93051
:108AC00089F404E110E00E94580C08E001BD839590
:108AD000833008F080E023EF3FE0082FA9010E94D7
:108AE000DC4AAECF9D3019F0AD3009F0A9CF21EFAF
:108AF0003FE0A9010E94D04A002331F000E021EFBD
:108B00003FE0A9010E94DC4A809BFECF04E110E017
:108B10000E94580C00E910E05ED326D3882391F41C
:108B200001E074D3902F0CE810E055D3092F0E9478
:108B3000C60E08E512E04FD301E0009358090E94E9
:108B4000D60EFDCF00914A09013059F101E00093A2
:108B50004A0920914A0914E00EEFEFD405E912E02A
:108B60003AD300E814E82EE130E040914A0950E0A1
:108B700060E070E04F5F5F4F6F4F7F4F0E94794B17
:108B80000E94A90D00EB12E026D300914A0920E0D3
:108B900030E0A9010E94DC4A09B904EF11E00E940B
:108BA000580C01E033D3902F0CE810E014D3092FB8
:108BB0000E94C60E08E512E00ED307E000935809A4
:108BC00001E010E0E8ECFCE0008311830E94012149
:108BD000E5EAFDE020813181273302E0300730F003
:108BE00023E333E012E20EEFB0D405C02FEF33E001
:108BF00012E20EEFAAD4813071F401E010E0E8EC4B
:108C0000FCE0008311830E94F52103E000935809E2
:108C10000E94692312C0823081F402E00093580957
:108C200000E00E94BC3E04E610E00E94580C04E103
:108C300010E00E94580C08E001BDFFCFFA93EA93C0
:108C40004A933A932A931A930A933FB74BB700E09B
:108C50000BBFAA9820919C000091ED0C10E00F70C2
:108C60001070F801E151F34F2083EDEEFCE000813C
:108C7000039500834BBF3FBF099119912991399109
:108C80004991E991F9911895FA93EA934A933A93A5
:108C90002A931A930A933FB74BB700E00BBF00919A
:108CA0005609102F1395109356092CB110E0F801B6
:108CB000E857F94F20834BBF3FBF09911991299184
:108CC00039914991E991F9911895AA98A99808EADA
:108CD00010E081D223C00E94B20E0E947D0D5E9AE8
:108CE0000091EE0C1091ED0C0117A9F75E9BFECFE1
:108CF0001A981B9A0091570910915609011771F0A3
:108D00000091570910E0F801E857F94F0081E7E5B5
:108D1000F9E01081139510830E94810D0091EE0CF3
:108D20001091ED0C011731F31B981A9AD9CF0E94BC
:108D3000A94B902F44249F3F29F400E91FE521E02F
:108D400030E004C008EE13E020E030E080E013C023
:108D50004091570950E0FA01E857F94F4081E7E5A3
:108D6000F9E0508153955083682F70E0FB01E65F76
:108D7000F74F408383958917D8F440E050E060E0D6
:108D800070E00090570910905609011479F40A0117
:108D90001B01A001B1014F5F5F4F6F4F7F4F001567
:108DA00011052205330568F744244394442081F2D9
:108DB000A82FB0E00091C0080E3F09F470C0442015
:108DC00071F09F3F61F0E8E5F9E0008100FF03C02A
:108DD0000FE11DE000D20091560900935709A4301D
:108DE00008F45DC000910A080F3F21F400910B08C0
:108DF0000F3F71F0E8E5F9E0008100FF03C004E3F4
:108E00001DE0E9D1009156090093570900E048C0E0
:108E100000910C081091C008011771F0E8E5F9E025
:108E2000008100FF03C00AE41DE0D5D1009156097E
:108E30000093570900E034C020910D0830E00A2F5C
:108E400010E0045010402017310771F0E8E5F9E018
:108E5000008100FF03C000E61DE0BDD1009156096E
:108E60000093570900E01CC082E007C090E0FC01BD
:108E7000E65FF74F0081B00F83958A17B8F3BF3FC5
:108E800071F0E8E5F9E0008100FF03C006E71DE0AE
:108E9000A2D1009156090093570900E001C00A2FA2
:108EA000E5E00C94B84B0E94AA4B3FEF3093BE080C
:108EB0003FEF3093BF080093C008022F0E5F00936E
:108EC000C1081093C20880E00DC090E0FC01E85793
:108ED000F84F0081A82FB0E01596FD01E254F74F3E
:108EE00000838395821788F300E02A5FA22F82E037
:108EF00007C090E0FC01E254F74F1081010F839509
:108F000090E0EA2FF0E031978E179F0794F30095D9
:108F100090E0FC01E254F74F00831B981A9A80E01E
:108F200009C05E9A90E0FC01E254F74F00810E9474
:108F30007D0D83958A17A8F35E9BFECF1A981B9A26
:108F40000A2FE4E00C94B94B0E94AA4BD801922F4F
:108F5000992359F40091C0080E3F21F400EF11E06D
:108F60003AD103C001E112E036D180E00CC0082FF5
:108F700010E0FD01E00FF11F00810E94390E00E2B8
:108F80000E94810D8395891790F301E412E023D1AB
:108F9000092F0E94C60EE4E00C94B94B0E94A84B26
:108FA000802F912F422E01E00093CC0CB0E029C01D
:108FB00040E050E060E070E0F0E08A019B01A80131
:108FC000B9014F5F5F4F6F4F7F4F083EE3E01E07D1
:108FD000E0E02E07E0E03E0778F400915709109199
:108FE0005609011721F040E050E060E070E00F2FDB
:108FF000F02FF395053608F30091560900935709B1
:10900000B395B23008F04EC000915609009357094D
:10901000242D192F082F47DFA02F913061F48E3FA8
:1090200029F455245A9450925A0930C006E0502E23
:1090300050925A092BC0923039F45090890706E0BB
:10904000500E50925A0922C08E3FC1F08F3140F429
:10905000082F10E0F801E55AF64F0081023870F051
:10906000843680F08E3670F4082F10E004561040DD
:10907000F801E558F64F0081023820F4552450924B
:109080005A0910C006E0502E50925A09552009F492
:10909000B7CF052D4CDE00935A0900915A090515EA
:1090A00009F086CF00E00093CC0C00915A09051519
:1090B00009F443C00091C0080E3FF9F1E8E5F9E07A
:1090C000008100FF15C00DED1DE085D0082F0E9426
:1090D000C60E07EB10E07FD02A2F0EEB18E034DF2E
:1090E00009EC10E078D020915A090AE018E02CDF52
:1090F000E8E5F9E0008101FF1EC000E011E80E94F0
:10910000973E082F0E94390E00E20E94810D092F20
:109110000E94390E00E20E94810D009188070E9492
:10912000390E00E20E94810D009189070E94390EDC
:1091300000E20E94810D00E014C000915909002353
:1091400079F007EB10E047D02A2F0EEB18E0FCDE99
:1091500009EC10E040D020915A090AE018E0F4DE52
:1091600001E0E6E00C94B74B0BED10E034D000E8E2
:1091700014E82EE130E04091990050E060E070E0AA
:109180004F5F5F4F6F4F7F4F0E94794B0E94A90D39
:1091900000E20E94810D00EB12E01DD00CE20E9463
:1091A000810D05EE10E017D000E814E82EE130E064
:1091B00049B150E060E070E04F5F5F4F6F4F7F4F0D
:1091C0000E94794B0E94A90D00E20E94810D00EBE4
:1091D00012E001D00895EF97EF97A49720E001C027
:1091E0002395203A60F430E0F801E20FF31F449138
:1091F000FE0130E0E20FF31F4083442389F78E0124
:109200000E94A50EEF96EF96A49608950E94AA4B91
:10921000B02FBB2361F00CE810E0DDDF09E40E9411
:10922000810D04E40E94810D0AE30E94810D90E00B
:1092300020E011E00EEFB2DE00915A09002309F49C
:1092400089C0A0E00EC0843658F08E3648F420E085
:10925000082F10E004561040F801E558F64F20831F
:10926000A39500915A09A01708F074C00A2F10E0C6
:10927000F801E65FF74F00810F3F91F70A2F10E0EA
:109280000F5F1F4FF801E65FF74F00810F3F41F777
:109290000A2F10E00E5F1F4FF801E65FF74F808145
:1092A0000A2F10E00D5F1F4FF801E65FF74F0081B6
:1092B000023009F044C00A2F10E00E5F1F4FF80182
:1092C000E65FF74F408150E00A2F10E00D5F1F4F1F
:1092D000F801E65FF74F208130E0240F351F0A2F99
:1092E00010E00B5F1F4FF801E65FF74F008110E0C1
:1092F000020F131F0F3F20E0120709F58F3140F4D2
:1093000020E8082F10E0F801E55AF64F20830DC041
:10931000843658F08E3648F420E8082F10E00456C2
:109320001040F801E558F64F2083BB2331F0082F99
:109330000E94390E00E20E94810D939591CF8F31EA
:1093400008F081CF20E0082F10E0F801E55AF64F31
:10935000208386CF40EC50EE60E070E080E059C0A2
:1093600002E0809F8001212F220F220B322F040F59
:10937000151F261F371F0F5F1F4F2F4F3F4FF8013D
:10938000322F3BBF0690102D00E00BBF00E022E023
:10939000829F212C220C2208322C040E151E261E20
:1093A000371EF001322D3BBF069020E02BBF112469
:1093B000000E111E082F10E0000F111FF801EA57D0
:1093C000F64F00821182082F10E0000F111FF801E4
:1093D000EA57F64F20813181203000E4300769F0F0
:1093E000082F10E0000F111FF801EA57F64F2081F7
:1093F0003181203000E4300759F400E010E0282FDC
:1094000030E0220F331FF901EA57F64F0083118332
:1094100083958F3108F4A4CF80E010C014E2082FA8
:109420000E943E2E22E0829F20E0020E22E0121EC9
:10943000F001EA53F64F0083118383958F3180F555
:10944000082F10E0F801E55AF64F00810023A9F338
:1094500010E1082F4DD00068282F30E0F901E55ABF
:10946000F64F008315E0082F43D0002321F020E0C1
:1094700015E0082F62D018E1082F3AD0013071F6BC
:109480001EE1082F0E943E2E22E0829F20E0020E65
:1094900022E0121EF001EA53F64F00831183CDCF74
:1094A00084E620C0A82FB0E0A456B040FD01E558E6
:1094B000F64F00810023A9F010E1082F19D00068B1
:1094C000A82FB0E0A456B040FD01E558F64F008348
:1094D00015E0082F0DD0002321F020E015E0082F23
:1094E0002CD083958E36F0F2092FE4E00C94B94B22
:1094F0001093880711E01093890722E012E04EDDF7
:10950000002319F000910F0808950FEF08951093AC
:10951000880712E01093890722E012E03FDD002364
:1095200049F03091100820E000910F0810E0020F80
:10953000131F08950FEF1FEF0895109388072093CE
:10954000890722E013E02ADD089510938807122F7F
:1095500010938907232F30E020938A0723E013E03C
:109560001DDD08950FE30DBF05E00EBFC0E0D5E09F
:109570000E94C44B002311F00E94D64B00E00BBFA9
:109580000E94FD430E94F94B0C94F94BE199FECFE8
:1095900008954F5F5F4FFADF4EBB5FBBE09A0895BF
:1095A000FADF0DB308954F5F5F4F4EBB5FBBF8947A
:1095B000E29AE19A0FBE08950FB6E8DF0DBBF5CF32
:1095C0000024E8E0EA9532F0001F001C0416D0F3F6
:1095D000041AF8CF001F402D00950895002411248F
:1095E0000030010741F01695079510F4040E151E82
:1095F000440F551FF5CF002D112D08954A951AF0EF
:10960000000F111FFBCF08954A951AF01695079584
:10961000FBCF089500241124EFE0001F111F001C50
:10962000111C0416150610F0041A150AEA95AAF77B
:10963000001F111F402D512D009510950895309554
:109640002095109501951F4F2F4F3F4F089570950E
:109650006095509541955F4F6F4F7F4F089500245F
:10966000112422243324E02FE12BE22BE32B71F091
:10967000369527951795079520F4040E151E261E7E
:10968000371E440F551F661F771FEDCF002D112D7C
:10969000222D332D08954A952AF0000F111F221F05
:1096A000331FF9CF08950024112422243324E0E24B
:1096B000EA9592F0001F111F221F331F001C111C7E
:1096C000221C331C041615062606370688F3041AD6
:1096D000150A260A370AECCF001F111F221F331F5D
:1096E000402D512D622D732D0095109520953095AC
:1096F0000895FF2777231AF4F1600E94274B332344
:109700001AF4F0950E941F4B0E94534BF69510F4EB
:109710000E941F4BF69510F40C94274B0895AF93BD
:10972000BF93B12FA02F3BBFD895EF5FFF4F3F4FA7
:109730000D9241505040B9F74BBFBF91AF91089582
:10974000DA92CA92BA92AA929A928A927A926A9279
:109750005A924A92BA93AA939A938A930895DD846F
:10976000CC84BB84AA84998488847F806E805D8049
:109770004C80BB81AA8199818881F0E00FB6F89472
:10978000CE0FDF1F0FBE089501E0089520E002D044
:10979000E9F708952D9301501040202F212B0895B3
:1097A0003BBF27913BB7F6DFD9F7089503E418E9EB
:1097B0002801F20130E03BBF07911691F201329689
:1097C000A791B691F2013496479157916691242F53
:1097D000252B262B21F0FA01362FE2DF01C0D6DF40
:1097E00007E0400E00E0501EA2014135584908F341
:1097F000089500008895FECF141A1F24292E3338AF
:109800003D4D151B20252A2F343908080809090960
:1098100009090909090909090909090909090808BA
:10982000080808080808080808070700FF030205D9
:1098300004070609080B0A0D0C0F0E111013121560
:1098400014160048014005519800AB098806000035
:109850000049440050494E47004700474F004452DA
:1098600045534554005245534554005359535F578F
:10987000520041435400414354494F4E0052454722
:109880005F575200570057520057524954450053F2
:10989000594E435F5752005357520043414C5500B5
:1098A000444543004845580043414C440052000D94
:1098B0000A205B4349443A005D200052455400525F
:1098C000455455524E0052554E0048454C50005498
:1098D00000544F53530043494400544553540043EC
:1098E000484B0044454D4F004D4F4E49544F520098
:1098F0004241554400534541524348004C454400C1
:109900005343414E00555044415445004400445592
:109910004D500042414C414E4345004F4646004F9A
:109920004E004E414D4500434F50590050005041AC
:1099300047450042004245464F5245004E004E45C5
:10994000585400474F544F004D4F4E00524500525F
:109950004400524541440048004558495400534191
:10996000560053415645004E4557004D004D495253
:10997000524F520053455400504C41590049004940
:109980004E534552540044454C455445004D4F56A6
:09999000450053005354455000FA
:00000001FF
